:020000040000FA
:061000007EEF3AF0120041
:06100800E3EF25F01200E9
:0610180022EF08F01200B7
:06102A0002004A750000FF
:10103000990100006400000048750000B70E000030
:0410400002000000AA
:0C104400D8CFE4FFE0CFE4FFE46EDACF89
:10105000E4FFE2CFDAFFE9CFE4FFEACFE4FFF3CF2A
:10106000E4FFF4CFE4FFE652D9CFE6FFE1CFD9FFAA
:10107000040EE126020EDB6A030EDB6A9EA27ED31B
:101080009E920401D65101E1A1D0030E526E2D5063
:10109000EA6A510FE96E010EEA22EF50525C30E12C
:1010A0002D50E96EEA6AD890E936EA36690EE926EB
:1010B000010EEA22EECF52F0EFCF53F053C052F0C0
:1010C000536A5250D76E2D50E96EEA6AD890E936CD
:1010D000EA36690EE926010EEA22EECF52F0EFCF92
:1010E00053F05250D66EF28AF294D58E2D50EA6AA1
:1010F000510FE96E010EEA22040EEF6E2D502F6E95
:10110000020E526E2E50EA6A510FE96E010EEA226B
:10111000EF50525C49E12E50E96EEA6AD890E93608
:10112000EA36690EE926010EEA22EE50ED1009E1D9
:101130002E50EA6A510FE96E010EEA22010EEF6E9F
:1011400033D0080E2E5C0CE2070E2E14526E010EE8
:10115000525204E0E846FE0B5206FCE189121AD016
:10116000100E2E5C0CE2070E2E14526E010E52521F
:1011700004E0E846FE0B5206FCE18A120BD0070E93
:101180002E14526E010E525204E0E846FE0B520637
:10119000FCE18B122E50EA6A510FE96E010EEA2231
:1011A000030EEF6E2E502D6E2E2A060E2E5C02E1DF
:1011B000080E04D0130E2E5C03E1160E2E6E59D1CC
:1011C000180E2E5C01E055D12E6A53D10E0100514C
:1011D00001E14FD10E01012B0E01AC510E01015D59
:1011E00001E247D1016B0E01AA51EA6A320FE96EA2
:1011F0000E0EEA22EF500E01EA6AAD25E96EAE51FD
:10120000EA22EF6A79907B6A7A6A0E01AA2B0E01B4
:10121000AB510E01AA5D01E3AA6BAA51E96EEA6A1D
:10122000D890E936EA36020EE9260E0EEA22EE5092
:10123000ED1001E11ED1AA51E96EEA6AD890E936B3
:10124000EA364A0EE9260E0EEA22EECF52F0EFCF32
:1012500053F0AA51E96EEA6AD890E936EA36020EEE
:10126000E9260E0EEA22EECF54F0EFCF55F054509F
:10127000521802E15550531801E1BDD0AA51E96E50
:10128000EA6AD890E936EA364A0EE9260E0EEA22D4
:10129000EECF54F0EFCF55F0AA51E96EEA6AD8903C
:1012A000E936EA36020EE9260E0EEA22EE50545CCA
:1012B000526EEE505558536E020E52C0DBFF030EB5
:1012C00053C0DBFF020EDBCF52F0030EDBCF53F037
:1012D00053343BE252500008000E535436E2020EE3
:1012E000DBCF52F0030EDBCF53F0AA51E96EEA6A6E
:1012F000D890E936EA367A0EE9260E0EEA22EECFCB
:1013000054F0EFCF55F05250545C5350555857E2BB
:10131000AA51E96EEA6AD890E936EA367A0EE926E9
:101320000E0EEA22EECF52F0EFCF53F0AA51E96E43
:10133000EA6AD890E936EA36020EE9260E0EEA226B
:101340005250EE265350ED2256D0020EDBCF52F013
:10135000030EDBCF53F0526C531E000E5322AA51E2
:10136000E96EEA6AD890E936EA367A0EE9260E0E78
:10137000EA22EECF54F0EFCF55F05250545C535068
:1013800055581DE2AA51E96EEA6AD890E936EA3664
:101390007A0EE9260E0EEA22EECF52F0EFCF53F08E
:1013A000AA51E96EEA6AD890E936EA36020EE926D1
:1013B0000E0EEA225250EE5E5350ED5A1CD0AA5146
:1013C000E96EEA6AD890E936EA364A0EE9260E0E48
:1013D000EA22EECF52F0EFCF53F0AA51E96EEA6A5B
:1013E000D890E936EA36020EE9260E0EEA2252C0FD
:1013F000EEFF53C0EDFFAA51EA6A320FE96E0E0EFE
:10140000EA22EF500E01EA6AAD25E96EAE51EA22FA
:10141000120EEF6EF29E0E01AA51E96EEA6AD890A2
:10142000E936EA36020EE9260E0EEA22EECF52F037
:10143000EFCF53F053C052F0536A5250B66EAA51D8
:10144000E96EEA6AD890E936EA36020EE9260E0E0F
:10145000EA22EECF52F0EFCF53F05250B56EF00EBD
:10146000B4140009B46EF00EB4140909B46E798096
:10147000F28E000ED8802154000E22542EE2302A23
:10148000000E31222150305C2250315826E3306A60
:10149000316A030E255C1FE22350EA6A480FE96EA9
:1014A000010EEA2280CFEFFF2350EA6A4B0FE96E6C
:1014B000010EEA2281CFEFFF2350EA6A4E0FE96E58
:1014C000010EEA2282CFEFFF232A030E235C01E301
:1014D000236A252A02D0216A226A000ED880265467
:1014E000000E275419E22B50000816E2322A000E93
:1014F00033222650325C275033580EE3326A336A67
:10150000030E2A5C07E2282A030E285C01E3286AFE
:101510002A2A02D0266A276A2B5000080AE2346A77
:101520003450040DF328C26E9E9C9F9C9D8CC280FB
:10153000C2820101995101E11DD1DE6ADD6ADECF6F
:1015400052F0DDCF53F0040E525C000E535801E30D
:1015500011D1DECFE9FFDDCFEAFF010ED890E936E9
:10156000EA36E806FBE19A0EE926010EEA22EE5081
:10157000ED1001E1D3D0DECFE9FFDDCFEAFF010EB0
:10158000D890E936EA36E806FBE1AA0EE926010E14
:10159000EA22EE50ED1026E1D9CFE9FFDACFEAFFDB
:1015A000EE50ED1001E18180D9CFE9FFDACFEAFFFB
:1015B000010EEE1803E1ED5001E18182D9CFE9FF80
:1015C000DACFEAFF020EEE1803E1ED5001E181846B
:1015D000D9CFE9FFDACFEAFF030EEE1803E1ED50B1
:1015E00001E18186DECFE9FFDDCFEAFF010ED89071
:1015F000E936EA36E806FBE1AA0EE926010EEA2200
:10160000EECF52F0EFCF53F0DECFE9FFDDCFEAFFB0
:10161000010ED890E936EA36E806FBE19A0EE92693
:10162000010EEA22EECF54F0EFCF55F0545052188D
:1016300029E15550531826E1D9CFE9FFDACFEAFF67
:10164000EE50ED1001E18190D9CFE9FFDACFEAFF4A
:10165000010EEE1803E1ED5001E18192D9CFE9FFCF
:10166000DACFEAFF020EEE1803E1ED5001E18194BA
:10167000D9CFE9FFDACFEAFF030EEE1803E1ED5010
:1016800001E18196DECFE9FFDDCFEAFF010ED890C0
:10169000E936EA36E806FBE1AA0EE926010EEA225F
:1016A000EE2A000EEF22DECFE9FFDDCFEAFF010ECA
:1016B000D890E936EA36E806FBE1AA0EE926010EE3
:1016C000EA22EECF52F0EFCF53F0DECFE9FFDDCFCD
:1016D000EAFF010ED890E936EA36E806FBE1A20EF1
:1016E000E926010EEA22EECF54F0EFCF55F0545028
:1016F00052183AE15550531837E1DECFE9FFDDCFFC
:10170000EAFF010ED890E936EA36E806FBE1AA0EB8
:10171000E926010EEA22EE6AED6A26D0D9CFE9FF6A
:10172000DACFEAFFEE50ED1001E18190D9CFE9FF69
:10173000DACFEAFF010EEE1803E1ED5001E18192EC
:10174000D9CFE9FFDACFEAFF020EEE1803E1ED5040
:1017500001E18194D9CFE9FFDACFEAFF030EEE1859
:1017600003E1ED5001E18196DF2A010E01E2E7D6A7
:10177000DB2AE5D60401B35101E0B3079EAC2CD0BF
:101780009E9CC450566E576E566AC3500001561048
:10179000546E57C055F03450060DF3CF52F0F4CFCD
:1017A00053F0000E5226010E53222850020D5250C3
:1017B000F324E96E5350F420EA6E54C0EEFF55C096
:1017C000EDFF342A2B50345C02E39D9C05D034504D
:1017D000040DF328C26EC282F2A442D0D59EF294C8
:1017E000F29A040E526E2F50EA6A510FE96E010E02
:1017F000EA22EF50525C34E1080E2F5C0DE2070E36
:101800002F14526E010E525204E0E846FE0B5206AF
:10181000FCE1E81C89161CD0100E2F5C0DE2070EAF
:101820002F14526E010E525204E0E846FE0B52068F
:10183000FCE1E81C8A160CD0070E2F14526E010E24
:10184000525204E0E846FE0B5206FCE1E81C8B16FF
:101850002F50EA6A510FE96E010EEA22020EEF6E76
:10186000040EE15C02E2E16AE552E16EE552E7CF87
:10187000D9FFE552E5CFF4FFE5CFF3FFE5CFEAFF6F
:10188000E5CFE9FFE5CFDAFFE550E5CFE0FFE5CFB3
:10189000D8FF1000D9CFE6FFE1CFD9FF020EE12635
:1018A000896A92682B6A8A6A93688B6A94688C96B4
:1018B0008C9495969594928E0401010ED56F0E012D
:1018C000B769B869296A286A2A6A246A236A256A74
:1018D000216A226A266A276A306A316A326A336A62
:1018E000346ACA82CA80CA9CCA9ACA88CA96FA0E40
:1018F000CB6EDF6ADFCF49F00C0EE76E4918E8AE19
:1019000002D0E73402D0E750495C36E2010EDB6AD0
:10191000DBCF49F0030EE76E4918E8AE02D0E7349A
:1019200002D0E750495C26E2DFCF49F04A6A49BE5F
:101930004A68060E4A02F3CF4AF04902F3CF49F053
:10194000F4504A26000E4926010E4A22010EDBCF32
:101950004BF04C6A4BBE4C68D8904B364C364950D5
:101960004B24E96E4A504C20EA6EEE6AED6A010E95
:10197000DB2ACED7DF2ABED70401CF6BD06BCD6B6D
:10198000CE6BD16BD26BD36BD46B2D6A2E6A2F6A60
:10199000DF6ADFCF49F0180EE76E4918E8AE02D0D3
:1019A000E73402D0E750495C1BE2DFCFE9FFEA6A87
:1019B000E9BEEA68D890E936EA36690EE926010EF2
:1019C000EA22EE6AED6ADFCFE9FFEA6AE9BEEA6879
:1019D000510EE926010EEA22010EEF6EDF2AD9D759
:1019E000D586D59AD59CF294F29AF194D08ECA9469
:1019F0009D829F926EEC27F01EEC35F0F28EF28CF9
:101A0000CA84020EE15C02E2E16AE552E16EE5524F
:101A1000E7CFD9FF1200D9CFE6FFE1CFD9FF050EFE
:101A2000E126020EDB6A030EDB6A040EDB6AE3ECDE
:101A30001CF02550000809E2E2EC13F0242A030E02
:101A4000245C01E1246A2506F4D72A50000809E243
:101A500012EC14F0292A030E295C01E1296A2A06F6
:101A6000F4D7200E0501E76EA819E8AE02D0E734DE
:101A700002D0E750A85D01E2B7D16550020B01E04A
:101A8000B3D1400EE66E400EE66E020EE66E81ECBD
:101A900033F0E552E552E552E76E030EE7CFDBFF88
:101AA000DB50000801E324D1040EDB6A030EDB5097
:101AB000F36E040EDBCFF4FFF350F45C01E318D1B6
:101AC000040EDB50EA6A400FE96E020EEA22EFCF05
:101AD000DFFF0101F65141E10D0E496EDF50495C17
:101AE00005E00A0E4A6EDF504A5C37E1010EF66FE0
:101AF0000401CF51EA6A000FE96E030EEA220D0ECF
:101B0000EF6ECF2B010EDB6ACF51F36E010EDBCFF0
:101B1000F4FFF350F45C1CE2010EDBCFE9FFEA6A4C
:101B2000E9BEEA68000EE926030EEA22EF50E66EEF
:101B3000010EDBCFE9FFEA6AE9BEEA68B20EE926E8
:101B4000010EEA22E552E750EF6E010EDB2ADCD7E8
:101B5000D5D90401CF6BD06BBBD01B0EDF5C09E184
:101B6000F25107E1010EF26F1B0EF36FF46BF56B90
:101B7000AFD0F2050BE15B0EDF5C08E11B0EF35DFD
:101B800005E1F45103E15B0EF46FA2D0F20566E1CA
:101B9000410EDF5C63E11B0EF35D60E15B0EF45D03
:101BA0005DE1F36BF46BF56BF26B010EDB6ADBCF7F
:101BB000E9FFEA6AE9BEEA68000EE926030EEA22B6
:101BC000EF500D081CE0010EDBCFE9FFEA6AE9BE29
:101BD000EA68B20EE926010EEA22EF50E66E010E27
:101BE000DBCFE9FFEA6AE9BEEA68000EE926030EE8
:101BF000EA22E552E750EF6E010EDB2AD8D7010E3C
:101C0000DBCFCFF40401CF51EA6A000FE96E030E77
:101C1000EA22EF6A010E496E6F0E4A6E4B6A49C0A6
:101C2000E6FFE66E4BC0E6FFB5EC38F0E552E55254
:101C3000E552000EE66E030EE66EFE0E496E6E0E67
:101C40004A6E4B6A49C0E6FFE66E4BC0E6FFB5EC54
:101C500038F04C6E050EE15E4C503AD0080EDF5C59
:101C60001CE10401CF51000818E2CF07CF51EA6A06
:101C7000000FE96E030EEA22EF6AFB0E496E6E0E4C
:101C80004A6E4B6A49C0E6FFE66E4BC0E6FFB5EC14
:101C900038F0E552E552E5521BD00D0EDF5C18E03E
:101CA0000A0EDF5C15E0200EDF5C12E30101F36B2E
:101CB000F46BF56BF26B0401CF51EA6A000FE96E29
:101CC000030EEA22DFCFEFFF0101F66B0401CF2BF9
:101CD0000401CF51496E4A6A000E491806E1010E0F
:101CE0004A1803E12C86CF6BD06B040EDB2ADED6BC
:101CF0002C5001E178D02CA00FD0F50E496E6E0E5D
:101D00004A6E4B6A49C0E6FFE66E4BC0E6FFB5EC93
:101D100038F0E552E552E5522CA20FD0D60E496EAE
:101D20006E0E4A6E4B6A49C0E6FFE66E4BC0E6FF98
:101D3000B5EC38F0E552E552E5522CA40FD0BA0EBE
:101D4000496E6E0E4A6E4B6A49C0E6FFE66E4BC0A6
:101D5000E6FFB5EC38F0E552E552E5522CA60FD07F
:101D60009E0E496E6E0E4A6E4B6A49C0E6FFE66EE5
:101D70004BC0E6FFB5EC38F0E552E552E5522CA831
:101D80000FD07F0E496E6E0E4A6E4B6A49C0E6FF59
:101D9000E66E4BC0E6FFB5EC38F0E552E552E55291
:101DA0002CAC0FD05E0E496E6E0E4A6E4B6A49C067
:101DB000E6FFE66E4BC0E6FFB5EC38F0E552E552C3
:101DC000E5522CAE0FD0450E496E6E0E4A6E4B6A30
:101DD00049C0E6FFE66E4BC0E6FFB5EC38F0E552D1
:101DE000E552E5522C6A3FD8050EE15C02E2E16A59
:101DF000E552E16EE552E7CFD9FF1200D9CFE6FFF9
:101E0000E1CFD9FFE652CDC4DFFFDF2A400E496E95
:101E1000DF50495C01E1DF6A0401CE51DF5C01E182
:101E200022D80401CD51EA6A000FE96E020EEA22BF
:101E3000FE0EDBCFEFFFCD2B400ECD5D01E1CD6B74
:101E4000CE51CD5D01E12C84FE0EDBCF49F04A6A14
:101E500049BE4A6849C0F3FF4AC0F4FFE552E55263
:101E6000E7CFD9FF1200D9CFE6FFE1CFD9FFE65285
:101E70000401CD51CE5D3DE00501905105E079ECC6
:101E800034F0D4EC1DF0F8D70401CE51D880CD55F4
:101E900017E2CE51CD5DDF6EDFCFE6FFCE514A6A4D
:101EA000000F496E020E4A2249C0E6FF4AC0E6FF13
:101EB000E1EC33F0E552E552E552CDC4CEF417D053
:101EC000400ED880CE55DF6EDFCFE6FFCE514A6A96
:101ED000000F496E020E4A2249C0E6FF4AC0E6FFE3
:101EE000E1EC33F0E552E552E5520401CE6B79ECBA
:101EF00034F0E552E552E7CFD9FF1200D9CFE6FF23
:101F0000E1CFD9FF040EE126DE6ADD6A020EDB6A4C
:101F1000030EDB6A0401D051EA6A000FE96E030E7A
:101F2000EA22EF50E66EE66A0EEC3AF0E552E55230
:101F3000020EF3CFDBFF0401D02BD051496E4A6A69
:101F4000000E491804E1010E4A1801E1D06B020E9F
:101F5000DB50DE6EDD6AD051EA6A000FE96E030ED7
:101F6000EA22EF502C0836E0D051EA6A000FE96E01
:101F7000030EEA22EF500D082DE0D051EA6A000F5F
:101F8000E96E030EEA22EF50E66EE66A0EEC3AF0D6
:101F9000E552E552030EF3CFDBFF0401D02BD05105
:101FA000496E4A6A000E491804E1010E4A1801E11F
:101FB000D06B020EDBCF4BF04BC04CF04B6A030EE4
:101FC000DB5000014B24496E000E4C204A6E49C084
:101FD000DEFFDD6E000EDFCF3DF0010EDBCF3EF009
:101FE000320E3D1802E1530E3E1801E1B4D1430E0A
:101FF0003D1802E1510E3E1801E1AAD14B0E3D18E9
:1020000002E1430E3E1801E1A0D14C0E3D1802E161
:10201000420E3E1801E196D1440E3D1802E14E0EEB
:102020003E1801E18CD1490E3D1802E14E0E3E18DA
:1020300001E182D1420E3D1802E1510E3E1801E14C
:1020400078D14C0E3D1802E1510E3E1801E16ED1DF
:102050004C0E3D1802E1530E3E1801E164D14E0EC4
:102060003D1802E1510E3E1801E15AD14E0E3D18C5
:1020700002E1530E3E1801E150D1430E3D1802E13A
:10208000530E3E1801E146D14D0E3D1802E1450EBA
:102090003E1801E13CD1500E3D1802E1510E3E18B0
:1020A00001E132D1500E3D1802E1540E3E1801E11B
:1020B00028D1500E3D1802E1530E3E1801E11ED109
:1020C0004D0E3D1802E1530E3E1801E114D1470EAA
:1020D0003D1802E1500E3E1801E10AD1430E3D18B1
:1020E00002E1500E3E1801E100D1490E3D1802E117
:1020F000430E3E1801E1F6D0490E3D1802E1520EA2
:102100003E1801E1ECD0490E3D1802E1530E3E1895
:1021100001E1E2D0530E3D1802E1430E3E1801E109
:10212000D8D0530E3D1802E1520E3E1801E1CED038
:10213000530E3D1802E1530E3E1801E1C4D0530E78
:102140003D1802E1420E3E1801E1BAD0430E3D189F
:1021500002E1420E3E1801E1B0D0430E3D1802E10B
:10216000520E3E1801E1A6D04F0E3D1802E1420E7C
:102170003E1801E19CD0570E3D1802E14D0E3E186D
:1021800001E193D0520E3D1802E14D0E3E1801E1DF
:102190008AD0440E3D1802E1500E3E1801E181D074
:1021A0004F0E3D1802E1500E3E1801E177D0490E66
:1021B0003D1802E1500E3E186EE0580E3D1802E147
:1021C000540E3E1865E0540E3D1801E13E505EE0AD
:1021D000410E3D1801E13E5057E0560E3D1801E119
:1021E0003E5050E0490E3D1801E13E5049E04F0E8F
:1021F0003D1801E13E5042E0550E3D1802E1430E0C
:102200003E183AE0580E3D1802E1430E3E1831E008
:10221000430E3D1801E13E502AE0520E3D1801E107
:102220003E5023E0580E3D1802E1520E3E181AE0CF
:10223000030EDB5001E092D0020EDBCFE6FFE66A30
:10224000DBCFE6FFE66A220E496E6E0E4A6E4B6ADF
:1022500049C0E6FFE66E4BC0E6FFB5EC38F04C6EC9
:10226000070E9AD058EC17F099D0CED897D063D9F2
:1022700095D05AEC17F092D0CBD890D01ADA8ED0F5
:10228000A1DA8CD0BFDA8AD0CDDA88D009D986D04D
:1022900056EC17F083D0D5EC15F080D072EC16F028
:1022A0007DD09DDB7BD059DB79D019DB77D00EEC6C
:1022B00018F074D05CEC17F071D00CEC18F06ED004
:1022C00010EC18F06BD012EC18F068D014EC18F089
:1022D00065D016EC18F062D018EC18F05FD01AEC4C
:1022E00018F05CD01CEC18F059D01EEC18F056D049
:1022F000AFEC18F053D004EC29F050D0F6EC2AF0F3
:102300004DD0BEEC2AF04AD0A3EC2AF047D05CECCA
:102310002BF044D0BCEC27F041D0F6EC2BF03ED0B3
:1023200026EC2CF03BD040EC2CF038D052EC2CF0CA
:1023300035D06DEC2CF032D0D8EC2BF02FD0E9EC6E
:102340002BF02CD0D4EC18F029D0D9EC18F026D0F2
:102350008AEC2CF023D0A8EC35F020D0030EDBCF94
:10236000E6FFE66A020EDBCFE6FFE66A030EDBCF8E
:10237000E6FFE66A020EDBCFE6FFE66AFA0E496E7A
:102380006D0E4A6E4B6A49C0E6FFE66E4BC0E6FF33
:10239000B5EC38F04C6E0B0EE15E4C500401D051A0
:1023A000EA6A000FE96E030EEA22EF500D080DE015
:1023B0002C500BE1520E496E4A6ADF50491803E176
:1023C000DE52DD504A1801E02C8ECFC4D0F4040E4A
:1023D000E15C02E2E16AE552E16EE552E7CFD9FF46
:1023E00012000401D5510FE0B00E496E740E4A6E12
:1023F0004B6A49C0E6FFE66E4BC0E6FFB5EC38F02D
:10240000E552E552E55212004AEC0CF0F1EF11F002
:10241000D9CFE6FFE1CFD9FF030EE126E66AD9CF97
:10242000E6FFDACFE6FF010EE66E13EC1AF0E55296
:10243000E552E552E552E66AD950010FE66E000E0C
:10244000DA20E66E020EE66E13EC1AF0E552E55263
:10245000E552E5522C501AE1DF0417E1D950010F83
:10246000E96EDACFEAFFEE50ED100AE0010E496E98
:102470004A6ADB50491808E1020EDB504A1804E1B1
:10248000010EDBCFD5F401D02C8CABDF030EE15C69
:1024900002E2E16AE552E16EE552E7CFD9FF1200B0
:1024A000D9CFE6FFE1CFD9FF030EE126020EDB6AAA
:1024B000E66A1F0EE66E000EE66E030EE66E13EC85
:1024C0001AF0E552E552E552E552E66AD950020F9C
:1024D000E66E000EDA20E66E010EE66E13EC1AF0E0
:1024E000E552E552E552E5522C501BE1020EDB505D
:1024F0000CE11F50201003E1216A226A11D0CA8426
:102500001FC021F020C022F00BD01F50201003E18B
:10251000266A276A05D0CA841FC026F020C027F08B
:1025200060DF030EE15C02E2E16AE552E16EE55232
:10253000E7CFD9FF1200D9CFE6FFE1CFD9FF0A0ECE
:10254000E126E66AD9CFE6FFDACFE6FF010EE66EB6
:1025500013EC1AF0E552E552E552E552E66AD9501D
:10256000010FE66E000EDA20E66E010EE66E13EC49
:102570001AF0E552E552E552E552E66AD950020FEB
:10258000E66E000EDA20E66E010EE66E13EC1AF02F
:10259000E552E552E552E552E66AD950040FE66E7F
:1025A000000EDA20E66E010EE66E13EC1AF0E5522C
:1025B000E552E552E552E66AD950050FE66E000E87
:1025C000DA20E66E010EE66E13EC1AF0E552E552E3
:1025D000E552E552E66AD950060FE66E000EDA20A3
:1025E000E66E010EE66E13EC1AF0E552E552E55286
:1025F000E552E66AD950070FE66E000EDA20E66E65
:10260000010EE66E13EC1AF0E552E552E552E55282
:10261000E66AD950080FE66E000EDA20E66E010E6B
:10262000E66E13EC1AF0E552E552E552E552E66A21
:10263000D950090FE66E000EDA20E66E010EE66E46
:1026400013EC1AF0E552E552E552E552E66AD9502C
:10265000030FE66E000EDA20E66E010EE66E13EC56
:102660001AF0E552E552E552E5522C5018E1DF50E0
:10267000926E010EDB50936E020EDB50946E040ED0
:10268000DB50956E050EDB50966E030EDB500C088A
:1026900005E20C0EF36E030EF3CFDBFFA2DE0A0E93
:1026A000E15C02E2E16AE552E16EE552E7CFD9FF73
:1026B0001200D9CFE6FFE1CFD9FF020EE126E66A8C
:1026C000D9CFE6FFDACFE6FF010EE66E13EC1AF083
:1026D000E552E552E552E552E76E010EE7CFDBFF2A
:1026E0002C5066E1010EDB5002E1DF50896E010ED5
:1026F000E66ED9CFE6FFDACFE6FFE66E13EC1AF00E
:10270000E552E552E552E552E76E010EE7CFDBFFF9
:102710002C504EE1010EDB5002E1DF508A6E010EBB
:10272000E66ED9CFE6FFDACFE6FFE66E13EC1AF0DD
:10273000E552E552E552E552E76E010EE7CFDBFFC9
:102740002C5036E1010EDB5002E1DF508B6E010EA2
:10275000E66ED9CFE6FFDACFE6FFE66E13EC1AF0AD
:10276000E552E552E552E552E76E010EE7CFDBFF99
:102770002C501EE1010EDB5002E1DF508C6E010E89
:10278000E66ED9CFE6FFDACFE6FFE66E13EC1AF07D
:10279000E552E552E552E552E76E010EE7CFDBFF69
:1027A0002C5006E1010EDB5002E1DF508D6E19DE88
:1027B000020EE15C02E2E16AE552E16EE552E7CF2A
:1027C000D9FF12008450E66EE66A8350E66EE66A30
:1027D0008250E66EE66A8150E66EE66A8050E66EEA
:1027E000E66ADD0E496E6D0E4A6E4B6A49C0E6FF21
:1027F000E66E4BC0E6FFB5EC38F04C6E0D0EE15EB8
:102800004C501200B80E496E740E4A6E4B6A49C0A5
:10281000E6FFE66E4BC0E6FFB5EC38F0E552E55258
:10282000E5521200D9CFE6FFE1CFD9FFE652DF6AC9
:10283000DB0E496E6D0E4A6E4B6A49C0E6FFE66ECE
:102840004BC0E6FFB5EC38F0E552E552E552DF6AE1
:102850002B50DF5C30E2DFCF49F04A6A49BE4A685C
:10286000060E4A02F3CF4AF04902F3CF49F0F45082
:102870004A26000E4926010E4A222950020D4950CF
:10288000F324E96E4A50F420EA6EEECFE6FFEFCF74
:10289000E6FFD50E4B6E6D0E4C6E4D6A4BC0E6FFDB
:1028A000E66E4DC0E6FFB5EC38F04E6E050EE15E0B
:1028B0004E50DF2ACDD7B50E496E740E4A6E4B6A64
:1028C00049C0E6FFE66E4BC0E6FFB5EC38F0E552D6
:1028D000E552E552E552E552E7CFD9FF1200D9CFD4
:1028E000E6FFE1CFD9FF030EE126E66AD9CFE6FF86
:1028F000DACFE6FFE66E13EC1AF0E552E552E55248
:10290000E552E66AD950020FE66E000EDA20E66E56
:10291000010EE66E13EC1AF0E552E552E552E5526F
:102920002C5011E1DECF49F0DDCF4AF0000E495CBA
:10293000100E4A5807E2DECFE9FFDDCFEAFF020EB4
:10294000DBCFEFFF4EDD030EE15C02E2E16AE55210
:10295000E16EE552E7CFD9FF1200D9CFE6FFE1CF14
:10296000D9FF030EE126E66AD9CFE6FFDACFE6FF0C
:10297000E66E13EC1AF0E552E552E552E5522C50A2
:1029800024E1DECF49F0DDCF4AF0000E495C100EA5
:102990004A5807E2DECFE9FFDDCFEAFF020EEFCFB4
:1029A000DBFF020EDBCFE6FFE66ACB0E496E6D0E53
:1029B0004A6E4B6A49C0E6FFE66E4BC0E6FFB5ECD7
:1029C00038F04C6E050EE15E4C50030EE15C02E205
:1029D000E16AE552E16EE552E7CFD9FF1200D9CFA7
:1029E000E6FFE1CFD9FF030EE126E66AD9CFE6FF85
:1029F000DACFE6FF050EE66E13EC1AF0E552E5526B
:102A0000E552E552E66AD950010FE66E000EDA2073
:102A1000E66E010EE66E13EC1AF0E552E552E55251
:102A2000E552E66AD950020FE66E000EDA20E66E35
:102A3000010EE66E13EC1AF0E552E552E552E5524E
:102A40002C5001E0A8D0020EDB50010801E2A0D01A
:102A5000010EDB50070801E29BD0410E496EDF50AA
:102A6000495C1AE1020EDB500CE1010EF36EDB5003
:102A700004E0D890F336E806FCE1F350F31C92161C
:102A800089D0010EF36EDB5004E0D890F336E806EF
:102A9000FCE1F35092127ED0420E496EDF50495C49
:102AA0001AE1020EDB500CE1010EF36EDB5004E084
:102AB000D890F336E806FCE1F350F31C93166AD085
:102AC000010EF36EDB5004E0D890F336E806FCE12B
:102AD000F35093125FD0430E496EDF50495C1AE108
:102AE000020EDB500CE1010EF36EDB5004E0D890D7
:102AF000F336E806FCE1F350F31C94164BD0010EBC
:102B0000F36EDB5004E0D890F336E806FCE1F350B6
:102B1000941240D0440E496EDF50495C1AE1020E17
:102B2000DB500CE1010EF36EDB5004E0D890F3367D
:102B3000E806FCE1F350F31C95162CD0010EF36E61
:102B4000DB5004E0D890F336E806FCE1F350951230
:102B500021D0450E496EDF50495C1AE1020EDB5070
:102B60000CE1010EF36EDB5004E0D890F336E8067A
:102B7000FCE1F350F31C96160DD0010EF36EDB5002
:102B800004E0D890F336E806FCE1F350961202D048
:102B90002C8C01D026DC030EE15C02E2E16AE552F6
:102BA000E16EE552E7CFD9FF1200D9CFE6FFE1CFC2
:102BB000D9FF030EE126020EDB6AE66AD9CFE6FFF3
:102BC000DACFE6FF050EE66E13EC1AF0E552E55299
:102BD000E552E552E66AD950010FE66E000EDA20A2
:102BE000E66E010EE66E13EC1AF0E552E552E55280
:102BF000E5522C506DE1010EDB50070854E3410E05
:102C0000496EDF50495C0BE1010EF36EDB5004E0CE
:102C1000D890F336E806FCE1F35080143FD0420E22
:102C2000496EDF50495C0BE1010EF36EDB5004E0AE
:102C3000D890F336E806FCE1F35081142FD0430E10
:102C4000496EDF50495C0BE1010EF36EDB5004E08E
:102C5000D890F336E806FCE1F35082141FD0440EFE
:102C6000496EDF50495C0BE1010EF36EDB5004E06E
:102C7000D890F336E806FCE1F35083140FD0450EEC
:102C8000496EDF50495C0FE1010EF36EDB5004E04A
:102C9000D890F336E806FCE1F3508414E76E020E98
:102CA000E7CFDBFF02D02C8C13D0DBCFE6FFE66A48
:102CB000C20E496E6D0E4A6E4B6A49C0E6FFE66E63
:102CC0004BC0E6FFB5EC38F04C6E050EE15E4C50A3
:102CD000030EE15C02E2E16AE552E16EE552E7CF04
:102CE000D9FF1200D9CFE6FFE1CFD9FF030EE126CD
:102CF000E66AD9CFE6FFDACFE6FF050EE66E93DB94
:102D0000E552E552E552E552E66AD950010FE66E0A
:102D1000000EDA20E66E010EE66E85DBE552E55226
:102D2000E552E552E66AD950020FE66E000EDA204F
:102D3000E66E010EE66E77DBE552E552E552E552AE
:102D40002C5001E0A9D0020EDB50010801E2A0D016
:102D5000010EDB50070801E29BD0410E496EDF50A7
:102D6000495C1AE1020EDB500CE1010EF36EDB5000
:102D700004E0D890F336E806FCE1F350F31C891622
:102D800089D0010EF36EDB5004E0D890F336E806EC
:102D9000FCE1F35089127ED0420E496EDF50495C4F
:102DA0001AE1020EDB500CE1010EF36EDB5004E081
:102DB000D890F336E806FCE1F350F31C8A166AD08B
:102DC000010EF36EDB5004E0D890F336E806FCE128
:102DD000F3508A125FD0430E496EDF50495C1AE10E
:102DE000020EDB500CE1010EF36EDB5004E0D890D4
:102DF000F336E806FCE1F350F31C8B164BD0010EC2
:102E0000F36EDB5004E0D890F336E806FCE1F350B3
:102E10008B1240D0440E496EDF50495C1AE1020E1D
:102E2000DB500CE1010EF36EDB5004E0D890F3367A
:102E3000E806FCE1F350F31C8C162CD0010EF36E67
:102E4000DB5004E0D890F336E806FCE1F3508C1236
:102E500021D0450E496EDF50495C1AE1020EDB506D
:102E60000CE1010EF36EDB5004E0D890F336E80677
:102E7000FCE1F350F31C8D160DD0010EF36EDB5008
:102E800004E0D890F336E806FCE1F3508D1202D04E
:102E90002C8C02D0F1EC11F0030EE15C02E2E16A4D
:102EA000E552E16EE552E7CFD9FF1200F1EF11F0E4
:102EB000F1EF11F0F1EF11F0D9CFE6FFE1CFD9FF3B
:102EC000040EE126E66AD9CFE6FFDACFE6FF050E6B
:102ED000E66EA9DAE552E552E552E552E66AD950C6
:102EE000010FE66E000EDA20E66E010EE66E9BDA4A
:102EF000E552E552E552E552E66AD950020FE66E18
:102F0000000EDA20E66E030EE66E8DDAE552E5522B
:102F1000E552E5522C5076E1D950020FE96EDACF36
:102F2000EAFF720ED880EE542E0EED5441E3D950D4
:102F3000020FE96EDACFEAFFEE50ED101FE04C68A9
:102F40004D684E6A2D0EE76E020EDBCF4FF0030E7A
:102F5000DBCF50F0E7504F26000E5022516A4F5001
:102F60004C5C496E50504D584A6E51504E584B6E05
:102F7000020E49C0DBFF030E4AC0DBFF010EDB502F
:102F8000070816E3410E496EDF50495C02E1DF6A33
:102F900011D0420E496EDF50495C02E1080E06D0A6
:102FA000430E496EDF50495C03E1100EDF6E02D024
:102FB0002C8C28D0010EDB50DF24E96EEA6AD89011
:102FC000E936EA36690EE926010EEA22020EDBCF67
:102FD000EEFF030EDBCFEDFF010EDB50DF24EA6ACC
:102FE000510FE96E010EEA22EF040AE1010EDB50F7
:102FF000DF24EA6A510FE96E010EEA22020EEF6E3B
:10300000F1EC11F0040EE15C02E2E16AE552E16EDE
:10301000E552E7CFD9FF1200F1EF11F0F1EF11F017
:10302000F1EF11F0F1EF11F0F1EF11F0F1EF11F01C
:10303000F1EF11F0F1EF11F0F1EF11F0D9CFE6FF60
:10304000E1CFD9FF070EE126E66AD9CFE6FFDACF56
:10305000E6FF030EE66EE7D9E552E552E552E5528A
:10306000E66AD950020FE66E000EDA20E66E030E15
:10307000E66ED9D9E552E552E552E5522C5065E1AC
:10308000DECF9AF1DDCF9BF1020EDBCFA2F1030E72
:10309000DBCFA3F1040EDB6A030EF36E040EDBCF6D
:1030A000F4FFF350F45C4FE2010EE66ED9CFE6FF79
:1030B000DACFE6FF030EE66EB6D9E552E552E552E9
:1030C000E552E76E050EE7CFDBFF010EE66ED95045
:1030D000020FE66E000EDA20E66E030EE66EA3D94E
:1030E000E552E552E552E552E76E060EE7CFDBFF0B
:1030F0002C502BE1050EDB5026E1060EDB5023E1C0
:10310000040EDB28E96EEA6AD890E936EA369A0EB0
:10311000E926010EEA22DECFEEFFDDCFEDFF040E41
:10312000DB28E96EEA6AD890E936EA36A20EE9268B
:10313000010EEA22020EDBCFEEFF030EDBCFEDFF26
:10314000040EDB2AA9D7F1EC11F0070EE15C02E2D4
:10315000E16AE552E16EE552E7CFD9FF1200D9CF1F
:10316000E6FFE1CFD9FFE652E66AD9CFE6FFDACF34
:10317000E6FF010EE66E57D9E552E552E552E552FB
:103180002C500DE1DF5007E0F00E9314936E010117
:10319000010E996F02D00101996BF1EC11F0E5522B
:1031A000E552E7CFD9FF1200F29EF29C0FEF00F03C
:1031B0001200D9CFE6FFE1CFD9FF100EE126E66A73
:1031C000D950010FE66E000EDA20E66EE66A2BD9C2
:1031D000E552E552E552E552E66AD9CFE6FFDACF8D
:1031E000E6FF010EE66E1FD9E552E552E552E552C3
:1031F000E66AD950040FE66E000EDA20E66E020E83
:10320000E66E11D9E552E552E552E552E66AD9502B
:10321000020FE66E000EDA20E66E030EE66E03D9AC
:10322000E552E552E552E552E66AD9500A0FE66EDC
:10323000000EDA20E66E060EE66EF5D8E552E5528F
:10324000E552E552E66AD950060FE66E000EDA2026
:10325000E66E070EE66EE7D8E552E552E552E55216
:10326000E66AD9500E0FE66E000EDA20E66E040E06
:10327000E66ED9D8E552E552E552E552E66AD950F4
:103280000F0FE66E000EDA20E66E050EE66ECBD866
:10329000E552E552E552E552010EDBCF49F04A6AAC
:1032A00049BE4A6849C0E6FF4AC0E6FFB60E4B6E0B
:1032B0006D0E4C6E4D6A4BC0E6FFE66E4DC0E6FFEC
:1032C000B5EC38F04E6E050EE15E4E50DFCFE6FFF6
:1032D000E66AAA0E496E6D0E4A6E4B6A49C0E6FF59
:1032E000E66E4BC0E6FFB5EC38F04C6E050EE15EC5
:1032F0004C50040EDBCFE6FF050EDBCFE6FF9E0E43
:10330000496E6D0E4A6E4B6A49C0E6FFE66E4BC0D1
:10331000E6FFB5EC38F04C6E050EE15E4C50020E47
:10332000DBCFE6FF030EDBCFE6FF920E496E6D0E9C
:103330004A6E4B6A49C0E6FFE66E4BC0E6FFB5EC4D
:1033400038F04C6E050EE15E4C50D9500A0FE96E14
:10335000DACFEAFFEECFE6FFEECFE6FFEECFE6FFF5
:10336000EFCFE6FF850E496E6D0E4A6E4B6A49C07F
:10337000E6FFE66E4BC0E6FFB5EC38F04C6E070E8C
:10338000E15E4C50D950060FE96EDACFEAFFEECF7E
:10339000E6FFEECFE6FFEECFE6FFEFCFE6FF780EDB
:1033A000496E6D0E4A6E4B6A49C0E6FFE66E4BC031
:1033B000E6FFB5EC38F04C6E070EE15E4C500E0E99
:1033C000DBCFE6FFE66A6C0E496E6D0E4A6E4B6A05
:1033D00049C0E6FFE66E4BC0E6FFB5EC38F04C6E38
:1033E000050EE15E4C500F0EDBCFE6FFE66A600E85
:1033F000496E6D0E4A6E4B6A49C0E6FFE66E4BC0E1
:10340000E6FFB5EC38F04C6E050EE15E4C50F1EC89
:1034100011F0100EE15C02E2E16AE552E16EE55264
:10342000E7CFD9FF1200D9CFE6FFE1CFD9FF090ED0
:10343000E126080EDB6A0D0E496E0401D051EA6ADE
:10344000000FE96E030EEA22EF50495C05E1FB0E26
:10345000DB5044E12C8842D0D051EA6A000FE96E7B
:10346000030EEA22EF502C081FE0FB0EDB501AE19E
:10347000D051EA6A000FE96E030EEA22EF50E66EC1
:10348000E66A390E496E6D0E4A6E4B6A49C0E6FF18
:10349000E66E4BC0E6FFB5EC38F04C6E050EE15E13
:1034A0004C502C8A020EE5D1D02BD051496E4A6A7D
:1034B000000E491804E1010E4A1801E1D06B0D0E0F
:1034C000496ED051EA6A000FE96E030EEA22EF500E
:1034D000495C06E1FB0EDB5001E12C88030EC9D1EB
:1034E0002D0E496ED051EA6A000FE96E030EEA22F2
:1034F000EF50495C2EE1040E4A6EFE0EDB504A5C32
:1035000028E0050E4B6EFE0EDB504B5C22E0FE0EFB
:10351000DB0401E147D1030E496EFE0EDB50495C2E
:1035200001E140D1070E4A6EFE0EDB504A5C01E11C
:1035300039D1010EF36E080EF3CFDBFFD02BD05143
:10354000496E4A6A000E491804E1010E4A1801E169
:10355000D06B040E496EFE0EDB50495C11E0050E87
:103560004A6EFE0EDB504A5C0BE00A0EE66ED9CFC7
:10357000E6FFDACFE6FF89D9E552E552E55242D0BF
:10358000D051EA6A000FE96E030EEA22EFCF49F04C
:10359000000E49C0DFFF010EDB6A020EDB6A030E7C
:1035A000DB6A050E496EFE0EDB50495C1FE1000E22
:1035B000DFCFE6FF010EDBCFE6FF0EEC3AF0E5527F
:1035C000E552F3CF49F0F4CF4AF04B6A4C6A4AAE69
:1035D00002D04B684C6849C0DFFF010E4AC0DBFFD8
:1035E000020E4BC0DBFF030E4CC0DBFF0401D02BEF
:1035F000D051496E4A6A000E491804E1010E4A187A
:1036000001E1D06B080EDB506FE0FE0EDB500FE1E6
:10361000D9CFE9FFDACFEAFFD880800EEE54000E52
:10362000EE54000EEE54000EEE5401E2BBD0020E3A
:10363000496EFE0EDB50495C0FE1D9CFE9FFDACFCE
:10364000EAFFD880000EEE54800EEE54000EEE54C9
:10365000000EEE5401E2A6D0060E4A6EFE0EDB50BE
:103660004A5C0FE1D9CFE9FFDACFEAFFD880000E3C
:10367000EE54000EEE54000EEE54800EEE5401E2B5
:1036800091D0D9CFE9FFDACFEAFF040EEECFDBFF0E
:10369000050EEECFDBFF060EEECFDBFF070EEECF03
:1036A000DBFF080EDB5001E196D0040EDBCF3BF0D0
:1036B000050EDBCF3CF0060EDBCF3DF0070EDBCF77
:1036C0003EF04068416842684368D6EC39F0040E29
:1036D00037C0DBFF050E38C0DBFF060E39C0DBFF4D
:1036E000070E3AC0DBFF77D0FE0EDB500EE1D9CFDC
:1036F000E9FFDACFEAFFD8807F0EEE54000EEE54D9
:10370000000EEE54000EEE544DE3FE0EDB040EE10F
:10371000D9CFE9FFDACFEAFFD880FF0EEE54000ED2
:10372000EE54000EEE54000EEE543CE3020E496ED1
:10373000FE0EDB50495C0EE1D9CFE9FFDACFEAFF9C
:10374000D880FF0EEE547F0EEE54000EEE54000EA5
:10375000EE5428E3030E4A6EFE0EDB504A5C0EE187
:10376000D9CFE9FFDACFEAFFD880FF0EEE54FF0E83
:10377000EE54000EEE54000EEE5414E3060E4B6EA3
:10378000FE0EDB504B5C11E1D9CFE9FFDACFEAFF47
:10379000D880FF0EEE54FF0EEE54FF0EEE547F0E57
:1037A000EE5403E22C8C010E64D0070E496EFE0E1F
:1037B000DB50495C10E0D9CFE9FFDACFEAFF040E15
:1037C000EECFDBFF050EEECFDBFF060EEECFDBFF0D
:1037D000070EEECFDBFFFE0EDB50070A38E0010AD2
:1037E00025E0050A16E0010A14E0030A08E0050ACC
:1037F00006E0010A04E0050A02E0040E3AD0FC0EDD
:10380000DBCFE9FFFD0EDBCFEAFF040EDBCFEFFFDE
:103810002FD0FC0EDBCFE9FFFD0EDBCFEAFF040E5D
:10382000DBCFEEFF050EDBCFEDFF22D0FC0EDBCFB2
:10383000E9FFFD0EDBCFEAFF040EDBCFEEFF050E46
:10384000DBCFEEFF060EDBCFEEFF070E0FD0FC0E38
:10385000DBCFE9FFFD0EDBCFEAFFDFCFEEFF010E8E
:10386000DBCFEEFF020EDBCFEEFF030EDBCFEEFF72
:10387000000E496E090EE15C02E2E16AE552E16E7A
:103880004950E552E7CFD9FF1200D9CFE6FFE1CF8B
:10389000D9FF020EE126FD0EDBCFE9FFFE0EDBCFE6
:1038A000EAFFEE6AEE6AEE6AEE6A010EDB6AFC0E71
:1038B000DB50F36E010EDBCFF4FFF350F45C62E2F9
:1038C0000401D051EA6A000FE96E030EEA22EFCF3D
:1038D000DFFF300EDF5C51E3DF5039084EE3FD0EB1
:1038E000DBCFE9FFFE0EDBCFEAFFEECF49F0EECFF4
:1038F0004AF0EECF4BF0EFCF4CF00A0E406E416A2B
:10390000426A436A49C03BF04AC03CF04BC03DF0BC
:103910004CC03EF0D6EC39F037C049F038C04AF020
:1039200039C04BF03AC04CF0300EDF5C4D6E4E6A41
:103930004F6A506AE85049264E504A224F504B2257
:1039400050504C22FD0EDBCFE9FFFE0EDBCFEAFF2D
:1039500049C0EEFF4AC0EEFF4BC0EEFF4CC0EEFF89
:103960000401D02BD051496E4A6A000E491807E174
:10397000010E4A1804E1D06B02D0000E04D0010EF3
:10398000DB2A95D7010E496E020EE15C02E2E16A84
:10399000E552E16E4950E552E7CFD9FF12002550BC
:1039A000E66EE66A2D0E496E6D0E4A6E4B6A49C090
:1039B000E6FFE66E4BC0E6FFB5EC38F04C6E050E48
:1039C000E15E4C5012000501A85108E0010E496E5D
:1039D0006550020B01E0010E495C1BE10101FA0791
:1039E000000EFB5BFC510BE1FA51FB1111E18C86DF
:1039F000A00EFA6F0F0EFB6F010EFC6F1200FA5152
:103A0000FB1163E18C96A00EFA6F0F0EFB6FFC6B3F
:103A10001200A80509E0020EA85D06E0040EA85DEC
:103A200003E0100EA85D1BE10101FA07000EFB5B2D
:103A3000FC510BE1FA51FB1111E18C86200EFA6F5B
:103A40004E0EFB6F010EFC6F1200FA51FB113DE1AF
:103A50008C96200EFA6F4E0EFB6FFC6B1200200E40
:103A6000A85D33E10101FA07000EFB5BFC510AE19E
:103A7000FA51FB112AE18C86100EFA6F270EFB6FAC
:103A8000010E18D0FC050AE1FA51FB111EE18C96DB
:103A9000100EFA6F270EFB6F020E0CD0020EFC5DAB
:103AA0000BE1FA51FB1111E18C86A00EFA6F860E24
:103AB000FB6F030EFC6F1200FA51FB1106E18C96AE
:0C3AC000100EFA6F270EFB6FFC6B12005B
:043ACC00D9CFE6FF69
:103AD000E1CFD9FFE652A098636A626A0F01160E21
:103AE000396F9F0E376F7B0E366F658C386B030E08
:103AF000E66EE66AE66A270EE66E0F0EE66E68EC84
:103B000038F0496E050EE15E4950659CDF6ADF5072
:103B1000496E4A6A100E495C000E4A5810E2DF50A6
:103B2000040DF3CFE9FFF4CFEAFF000EE926040EFF
:103B3000EA22EE6AEE6AEE6AEE6ADF2AE8D70F0141
:103B4000160E266F62A602D06296FCD70501C36BE3
:103B5000C86BC96BCA6B6598DF6A040EDF5C18E23C
:103B6000EA6ADF34FE0BEA36E96EB70EE926050E87
:103B7000EA22EE6AED6AEA6ADF34FE0BEA36E96EA3
:103B8000AF0EE926050EEA22EE6AED6ADF2AE5D7D6
:103B90000501080EB76F040EB86FA96BA86BE5524C
:103BA000E552E7CFD9FF1200D9CFE6FFE1CFD9FF29
:103BB000E65282BE06D0656A0F01366B0501A86B1E
:103BC0008AD00501A85110E1656A0F01366B160E07
:103BD000396F9F0E376F7B0E366F65B602D06586E4
:103BE000FCD70501010EA86FA8050AE165BA08D047
:103BF000626A0F01366B368136890501020EA86FA5
:103C00006250040B06E00F013651040B02E062948F
:103C1000BBD865B260D06250010B13E00F01365182
:103C2000010B0FE053DF0501040EA86F0401400EE5
:103C3000026F040E036F400E016F006B8C0E0013B9
:103C400062906250100B06E00F013651100B02E03B
:103C500088D862986250400B14E00F013651400B37
:103C600010E0010EE66EE66A000EE66EE66A730E7E
:103C7000E66EE66ACEEC37F0496E060EE15E49501C
:103C8000629C6250200B05E00F013651200B01E0D1
:103C90004ED86250020B14E00F013651020B10E0B7
:103CA000010EE66EE66A000EE66EE66AE6687F0ED4
:103CB000E66ECEEC37F0496E060EE15E4950636A5F
:103CC000040E0501E76EA819E8AE02D0E73402D071
:103CD000E750A85D02E2A19825D00F0136A721D0B8
:103CE000DF6A040EDF5C1DE262A61BD064CFD0F554
:103CF0006296780E0501D01502E15CD810D0000E56
:103D0000E66EE66AD00EE66E050EE66E720EE66EA2
:103D1000E66ACEEC37F0496E060EE15E4950DF2AC6
:103D2000E0D7A198E552E552E7CFD9FF12000F0185
:103D300026A115D0ABC5E9FFACC5EAFFEF5080085E
:103D40000DE1B7C5E9FFB8C5EAFFEF50840806E109
:103D5000ABC5E9FFACC5EAFF8C0EEF6E2691629A07
:103D600012000F01368562986582000EE66EE66AE3
:103D7000E66EE66A750EE66EE66ACEEC37F0496EE0
:103D8000060EE15E49501200000EE66EE66AE66E2F
:103D9000E66A740EE66EE66ACEEC37F0496E060E01
:103DA000E15E495065920F01369562A402D062949B
:103DB000FCD71200D9CFE6FFE1CFD9FFE652FD0EC6
:103DC0000501D0155AE17E0ED015E8407F0B040D99
:103DD000F3CFABF5F4CFACF5000EAB27040EAC235C
:103DE000ABC5ADF5ACC5AEF5AD75ABC5E9FFACC5C2
:103DF000EAFFEF503C0BE842E8420D083CE1ABC55E
:103E0000E9FFACC5EAFF020EE926000EEA22EECF7A
:103E100049F0EFCF4AF0480E49182BE1040E4A183A
:103E200028E1ABC5E9FFACC5EAFF020EE926000EAA
:103E3000EA22400EEE6E040EED6EDF6ADF50496E30
:103E40004A6A080E495C000E4A5813E2DF50EA6ADB
:103E5000480FE96E040EEA22EF50E66EDF50EA6A80
:103E6000400FE96E040EEA22E552E750EF6EDF2ABA
:103E7000E5D70DD807D02ED805D0FD0ED0150408F3
:103E800001E14ED8E552E552E7CFD9FF1200B7C5A0
:103E9000E9FFB8C5EAFFEF50800B05E0B7C5E9FFC1
:103EA000B8C5EAFFEF6A0501BF6BC06BC46BC56B99
:103EB000C36BB5D8000EE66EE66AE66EE66A030EE0
:103EC000E66EE66ACEEC37F0496E060EE15E4950CA
:103ED000AAEF21F0020E0501C05D02E105EF23F01B
:103EE0006CD80501D1511AE1ADC5E9FFAEC5EAFFB5
:103EF000EE52400EEF6EADC5E9FFAEC5EAFF020E11
:103F0000E926000EEA22400EEE6E040EED6EADC5FF
:103F1000E9FFAEC5EAFF8C0EEF6E1200D16B120006
:103F2000D9CFE6FFE1CFD9FFE652B7C5E9FFB8C563
:103F3000EAFFEF50400B01E0010EDF6E0501B7759F
:103F4000080EA85D0CE142C438FF0F01385100088B
:103F500003E20501100E02D00501040EA86FC00592
:103F600026E1B7C5E9FFB8C5EAFF020EE926000E53
:103F7000EA22480EEE6E040EED6EBEDA020E050168
:103F8000BF5D06E1B7C5E9FFB8C5EAFF840E0DD0F5
:103F9000DF5006E1B7C5E9FFB8C5EAFFC80E05D096
:103FA000B7C5E9FFB8C5EAFF880EEF6E01D005D8A6
:103FB000E552E552E7CFD9FF1200D9CFE6FFE1CFB6
:103FC000D9FF020EE1260501C06BB7C5E9FFB8C5F0
:103FD000EAFFEF6A040EB719496EB8C54AF0DE6E03
:103FE000B8C5DDFFDECFE9FFDDCFEAFFEF6AC8AF7E
:103FF0000CD0CB51CC1107E005D0CCC5FAFF0501A0
:10400000CB51F96EFADF0501C89F020EE15C02E2B6
:10401000E16AE552E16EE552E7CFD9FF12000401F3
:104020004051600BE842E842E842E842E8420009B9
:1040300001E0120041510C0A50E00B0A3FE00C0A6B
:1040400031E0010A22E00B0A1EE0020A1CE0030A2A
:1040500018E0080A10E0010A0CE00F0A08E0030A61
:1040600001E012000501C38F080EA86F1200F3EFE4
:1040700020F0A1EF23F00501A90EC16F050EC26F5C
:104080000CD050EF21F06EEF20F044510501C16FCC
:10409000C26BAA0EC127050EC223C381010EC46FD5
:1040A000C38F12000501C38F04014451EA6AAA0FAD
:1040B000E96E050EEA2242C4EFFF1200000EE66E22
:1040C000E66AE66EE66A020EE66EE66ACEEC37F067
:1040D000496E060EE15E495012001200D9CFE6FF8C
:1040E000E1CFD9FF040EE1260401420510E1405161
:1040F0001F0B00090CE10501C38F030E0401415D94
:1041000004E10501010ECF6F02D00501CF6B040160
:1041100042515FE140511F0B02085BE144510F0B1C
:10412000000957E00501C38F040144BF0BD044517F
:104130000F0BE96EEA6AD890E936EA36AF0EE92647
:10414000050E0AD044510F0BE96EEA6AD890E936A1
:10415000EA36B70EE926050EEA22EECFDEFFEDCFF6
:10416000DDFF030E415D06E1DECFE9FFDDCFEAFFB3
:10417000840E2ED044510F0B4A6A260F496E0F0E43
:104180004A22020E49C0DBFF030E4AC0DBFF020ECB
:10419000DBCFE9FF030EDBCFEAFFEF9044AF0CD09B
:1041A000DECFE9FFDDCFEAFFEF6ADF74DECFE9FFA4
:1041B000DDCFEAFF400E0CD0DECFE9FFDDCFEAFF16
:1041C000880EEF6EDF74DECFE9FFDDCFEAFFC80EA9
:1041D000EF6E040EE15C02E2E16AE552E16EE55247
:1041E000E7CFD9FF1200800E0401405D58E10501C0
:1041F000C00EC36F04014351030A2FE0010A09E016
:10420000030A4BE10501980EC16F720EC26F120EC8
:104210003ED04251F66EF76AD890F636F7361F0E4A
:10422000F626730EF7220900F5CFC1F50A00F5CF87
:10423000C2F5020E0501F76AC125F66EC251F722DA
:104240000800F5CFC4F5030EF76AC125F66EC2511A
:10425000F7220800F5CFC5F51200030E425D1AE201
:104260004251F66EF76AD890F636F736210EF626EA
:10427000730EF7220900F5CFC1F50A00F5CFC2F59C
:10428000C1C5F6FFC2C5F7FF0800F5500501C46FB0
:10429000C56B12000501C36B12000501C36B120050
:1042A000D9CFE6FFE1CFD9FF020EE1260401486B2A
:1042B000496B40511F0B020A11E0030A0CE0010A8E
:1042C00035E10501C38F040148810501CF052EE1C9
:1042D000040148832BD00501C38F28D00501C38F6B
:1042E000040144BF0BD044510F0BE96EEA6AD89029
:1042F000E936EA36AF0EE926050E0AD044510F0B17
:10430000E96EEA6AD890E936EA36B70EE926050E74
:10431000EA22EECFDEFFEDCFDDFFDECFE9FFDDCF1E
:10432000EAFFEF50040B02E0010E486F0501C3AF36
:1043300007D0480EC16F040EC26FC381020EC46F56
:10434000020EE15C02E2E16AE552E16EE552E7CF7E
:10435000D9FF120065980501C3BF47D0C8AF26D06A
:10436000020EC06FB7C5E9FFB8C5EAFFEE52EF6AAB
:10437000B7C5E9FFB8C5EAFFC80EEF6EADC5E9FFE6
:10438000AEC5EAFFEE52400EEF6EADC5E9FFAEC519
:10439000EAFF020EE926000EEA22480EEE6E040E37
:1043A000ED6EADC5E9FFAEC5EAFF7AD0ADC5E9FF58
:1043B000AEC5EAFFEE52400EEF6EADC5E9FFAEC5E9
:1043C000EAFF020EE926000EEA22400EEE6E040E0F
:1043D000ED6EADC5E9FFAEC5EAFF8C0EEF6EB7C559
:1043E000E9FFB8C5EAFF840E5CD0C8BF84D00401E1
:1043F00040AF59D00501C4510401465D0501C551C6
:104400000401475904E246C4C4F547C4C5F574D84D
:104410000501010EC06FADC5E9FFAEC5EAFFEE5262
:10442000400EEF6EADC5E9FFAEC5EAFF020EE9260C
:10443000000EEA22400EEE6E040EED6EADC5E9FFF1
:10444000AEC5EAFF800EEF6ED16BABC5E9FFACC520
:10445000EAFFEE52400EEF6EABC5E9FFACC5EAFFD6
:10446000020EE926000EEA22400EEE6E040EED6EFC
:10447000ABC5E9FFACC5EAFF840EEF6E010ED16F4C
:10448000B7C5E9FFB8C5EAFF020EE926000EEA2229
:10449000480EEE6E040EED6EB7C5E9FFB8C5EAFF33
:1044A000C80EEF6E12000501020EC06FB7C5E9FF1E
:1044B000B8C5EAFFEE52EF6AB7C5E9FFB8C5EAFF33
:1044C000C80EEF6EADC5E9FFAEC5EAFFEE52400E75
:1044D000EF6EADC5E9FFAEC5EAFF020EE926000E9C
:1044E000EA22480EEE6E040EED6EADC5E9FFAEC5D4
:1044F000EAFFC80EEF6E1200D9CFE6FFE1CFD9FF79
:10450000020EE1260501400EC45D000EC5590DE204
:10451000C4C5DEFFC5C5DDFFBF5102E1010E03D0FA
:10452000BF0506E1020EBF6F03D0400EDE6EDD6AEE
:10453000B7C5E9FFB8C5EAFFEF92B7C5E9FFB8C54F
:10454000EAFFEF90B7C5E9FFB8C5EAFF010EDB50FF
:10455000EF12B7C5E9FFB8C5EAFFEE52DFCFEFFFB4
:10456000000EDB50C45F010EDB50C55B480ECD6F03
:10457000040ECE6FC3B120D0D9CFE9FFDACFEAFF66
:10458000EE50ED1038E0C1C5F6FFC2C5F7FFC12BF4
:10459000000EC2230800F550E66ECDC5E9FFCEC57A
:1045A000EAFFCD2B000ECE23E552E750EF6EDF067B
:1045B000010EE2E2DB06E0D7D9CFE9FFDACFEAFF6E
:1045C000EE50ED1018E0C1C5E9FFC2C5EAFFC12BEE
:1045D000000EC223EF50E66ECDC5E9FFCEC5EAFF5F
:1045E000CD2B000ECE23E552E750EF6EDF06010E15
:1045F000E3E2DB06E1D7020EE15C02E2E16AE552AA
:10460000E16EE552E7CFD9FF1200D9CFE6FFE1CF47
:10461000D9FF020EE126ABC5E9FFACC5EAFFEE52B9
:10462000EFCFDFFFDFCF49F049500501C95D000E34
:10463000CA5902E2C9C5DFFFDF50496E4A6AE85035
:10464000C95DC96F4A50CA59CA6F010EDB6ADF5093
:10465000F36E010EDBCFF4FFF350F45C16E2010EB3
:10466000DB50EA6A480FE96E040EEA22EF50E66E6C
:10467000C6C5E9FFC7C5EAFFC62B000EC723E55232
:10468000E750EF6E010EDB2AE2D7000ED880C95545
:10469000000ECA5527E2ADC5E9FFAEC5EAFFEE52EE
:1046A000400EEF6EADC5E9FFAEC5EAFF020EE9268A
:1046B000000EEA22480EEE6E040EED6EABC5E9FF69
:1046C000ACC5EAFFEF50400B06E1ADC5E9FFAEC552
:1046D000EAFFC80E05D0ADC5E9FFAEC5EAFF880EFA
:1046E000EF6E25D0ADC5E9FFAEC5EAFFEE52400E34
:1046F000EF6EADC5E9FFAEC5EAFF020EE926000E7A
:10470000EA22400EEE6E040EED6EADC5E9FFAEC5B9
:10471000EAFF840EEF6ECB51CC1107E005D0CCC57B
:10472000FAFF0501CB51F96EFADF0501C89F020EB1
:10473000E15C02E2E16AE552E16EE552E7CFD9FFC2
:104740001200D9CFE6FFE1CFD9FFE6520501C38FB2
:10475000030EE66EE66AE66A270EE66E0F0EE66E5A
:1047600068EC38F0496E050EE15E4950DF6ADF50B3
:10477000496E4A6A100E495C000E4A5810E2DF503A
:10478000040DF3CFE9FFF4CFEAFF000EE926040E93
:10479000EA22EE6AEE6AEE6AEE6ADF2AE8D7658CF4
:1047A000010EE66EE66AE66AAA0EE66E050EE66E93
:1047B00068EC38F0496E050EE15E4950659C0501D4
:1047C000080EB76F040EB86F000EAB6F040EAC6F1F
:1047D000ABC5ADF5AE6F42C4A9F5A95102E1100E0B
:1047E00012D0010EE66EE66AA90EE66E050EE66EC2
:1047F000010EE66EE66ACEEC37F0496E060EE15E1B
:1048000049500501200EA86FE552E552E7CFD9FFC8
:104810001200D9CFE6FFE1CFD9FF020EE126000E4C
:10482000DE6E040EDD6EFD0EDB50E8244B6EFE0ED8
:10483000DB50040DF3504B24040DF350496E4A6ACB
:10484000020E0F0B05E0D8904A324932E806FBE130
:10485000D89049364A36D89049364A36D9CFE9FFFA
:10486000DACFEAFF4950EE264A50ED22DECFE9FFCB
:10487000DDCFEAFFEF9EFD0EDB500AE1FE0EEA6A95
:10488000DB34FE0BEA36E96EAF0EE926050E09D0E1
:10489000FE0EEA6ADB34FE0BEA36E96EB70EE92655
:1048A000050EEA22DECFEEFFDDCFEDFFDECFE9FF22
:1048B000DDCFEAFFEF9CDECFE9FFDDCFEAFF040E9C
:1048C000E926000EEA22EF8C020EE15C02E2E16AC8
:1048D000E552E16EE552E7CFD9FF1200D9CFE6FFEE
:1048E000E1CFD9FF020EE126FE0EDB504A6A260F09
:1048F000496E0F0E4A2249C0DEFF4AC0DDFFDECFFF
:10490000E9FFDDCFEAFFFD0EDBCFEFFFDBA407D031
:10491000E66AFE0EDBCFE6FF7CDFE552E552FD0ED8
:10492000DBA208D0010EE66EFE0EDBCFE6FF71DFE4
:10493000E552E552020EE15C02E2E16AE552E16E07
:10494000E552E7CFD9FF1200D9CFE6FFE1CFD9FF7B
:10495000020EE126FE0EDB5020E1ADC5E9FFAEC53B
:10496000EAFFEE52400EEF6EADC5E9FFAEC5EAFFBD
:10497000020EE926000EEA22400EEE6E040EED6EE7
:10498000ADC5E9FFAEC5EAFF8C0EEF6EB7C5E9FF16
:10499000B8C5EAFF840EEF6E3BD0FD0EDB50E82475
:1049A0004B6EFE0EDB50040DF3504B24040DF3CF81
:1049B00049F0F4CF4AF0000E4926040E4A2249C0BD
:1049C000DEFF4AC0DDFF840EDECFE9FFDDCFEAFF68
:1049D000E850EF12FD0EDB50E8244B6EFE0EDB506C
:1049E000040DF3504B24010F040DF3CF49F0F4CF25
:1049F0004AF0000E4926040E4A2249C0DEFF4AC092
:104A0000DDFF840EDECFE9FFDDCFEAFFE850EF12D5
:104A1000020EE15C02E2E16AE552E16EE552E7CFA7
:104A2000D9FF1200D9CFE6FFE1CFD9FF020EE12670
:104A3000FD0EDB500AE0FE0EEA6ADB34FE0BEA36BE
:104A4000E96EB70EE926050E09D0FE0EEA6ADB34E0
:104A5000FE0BEA36E96EAF0EE926050EEA22EECF2E
:104A6000DEFFEDCFDDFFD9CFE9FFDACFEAFFEE5071
:104A7000ED1003E1F36AF46A44D0DECFE9FFDDCF45
:104A8000EAFF020EE926000EEA22FB0EDBCFEEFF64
:104A9000FC0EDBCFEDFFDECFE9FFDDCFEAFFEE520C
:104AA000FA0EDBCFEFFF400EDECFE9FFDDCFEAFFEE
:104AB000E850EF16880EDECFE9FFDDCFEAFFE850C1
:104AC000EF12FD0EDB500AE0FE0EEA6ADB34FE0B4D
:104AD000EA36E96EB70EE926050E09D0FE0EEA6A3F
:104AE000DB34FE0BEA36E96EAF0EE926050EEA224C
:104AF000EF74DECF49F0DDCF4AF049C0F3FF4AC082
:104B0000F4FF020EE15C02E2E16AE552E16EE55279
:104B1000E7CFD9FF1200D9CFE6FFE1CFD9FF65A8D3
:104B20004ED0FE0EEA6ADB34FE0BEA36E96EB70EB3
:104B3000E926050EEA22EE50EFCFEAFFE96E400EBD
:104B4000EE16EE6AEE6AEE6AFE0EEA6ADB34FE0BE1
:104B5000EA36E96EB70EE926050EEA22EE50EFCFEF
:104B6000EAFFE96EEE7CFE0EEA6ADB34FE0BEA3603
:104B7000E96EB70EE926050EEA22EF74400E496E83
:104B8000FE0EEA6ADB34FE0BEA36E96EB70EE92662
:104B9000050EEA22EE50EFCFEAFFE96E4950EF161C
:104BA000FE0EEA6ADB34FE0BEA36E96EB70EE92642
:104BB000050EEA22EE50EFCFEAFFE96EEF7CE552F8
:064BC000E7CFD9FF12004F
:0A4BC600DACFE4FFE2CFDAFFE9CF17
:104BD000E4FFEACFE4FFE6529EA078D19E908E0ECD
:104BE000CE6ECF681850196E1A6A010E1B6E020E37
:104BF0001E5C0EE104019C519D1104E004019C0720
:104C0000000E9D5B04019C519D1101E01B6A06D1C1
:104C10001E0401E097D0105011100AE11250131039
:104C200007E11450151004E11650171001E189D066
:104C30000401A5510BE018A202D08C8E01D08C9EED
:104C400018A602D08C8A01D08C9A0AD018A202D061
:104C50008C8E01D08C9E18A602D08C8A01D08C9AA2
:104C6000105011101DE000500824006E0150092062
:104C7000016E000ED8800054800E015410E200C076
:104C800000F001C001F0000E005E800E015A010E1E
:104C90001910196E010E1A6E1006000E115A1B6AB9
:104CA000125013101DE002500A24026E03500B2014
:104CB000036E000ED8800254800E035410E202C02E
:104CC00002F003C003F0000E025E800E035A040ED1
:104CD0001910196E010E1A6E1206000E135A1B6A75
:104CE0001A502FE00401A55105E019B08B8219B4C8
:104CF0008C8804D019B08B8219B48C880000000015
:104D000000000000000000000000000000000000A3
:104D10000000000000000000000000000000000093
:104D20000000000000000000000000000000000083
:104D300000000401A55103E08B928C9802D08B9265
:104D40008C986CD0030E1E5C33E10401D65105E053
:104D5000A9C47BF1AAC47CF119D00E01005114E062
:104D6000B3CE7AFEB4CE7BFEB1CE4AFEB2CE4BFEBF
:104D70000E01040E326F0E010251031104E1B1CE97
:104D800002FEB2CE03FE02D00401A26B8A98040197
:104D90009C519D1104E004019C07000E9D5B0401E1
:104DA0009C519D1101E01B6A0401010EAB6F36D0CE
:104DB000040E1E5C33E10401D65105E0A7C47BF16B
:104DC000A8C47CF11AD00E01005114E0B5CE7AFED1
:104DD000B6CE7BFEAFCE4AFEB0CE4BFE0E01040E29
:104DE000326F0E010251031104E1AFCE02FEB0CECC
:104DF00003FE03D00401010EA26F8A8804019C51B6
:104E00009D1104E004019C07000E9D5B04019C5170
:104E10009D1101E01B6A0401AB6B00D01B504AE0FE
:104E20001E6A1D5047E01C6A040E1C5C3AE21C50CE
:104E3000E96EEA6AD890E936EA36880EE926040E69
:104E4000EA22EECF58F0EFCF59F01C50E96EEA6A33
:104E5000D890E936EA36080EE926000EEA2258C054
:104E6000EEFF59C0EDFF1C50E96EEA6AD890E936B2
:104E7000EA36900EE926040EEA22EECF58F0EFCF84
:104E800059F01C50E96EEA6AD890E936EA36100EFD
:104E9000E926000EEA2258C0EEFF59C0EDFF1C2A99
:104EA000C3D798C418F099C41EF09AC49CF49BC44C
:104EB0009DF41D6A8050800B06E00401B25106E0AB
:104EC0008150010B03E10401010EB16FE552E5CF02
:104ED000EAFFE5CFE9FFE5CFDAFF1100010E086E2A
:104EE000096A0A6E0B6A0C6E0D6A0E6E0F6A106A02
:104EF000116A126A136A146A156A166A176A1D6AB9
:104F0000CD92CD9ECD9CCD8ACD98CD96CD948E0E52
:104F1000CE6ECF68CD809F809E909D8092800F0145
:104F2000FE0E486F170E496F8D8496948D8296926F
:104F3000898C929C8D8096908C8C959C8B9294926F
:104F40008C9E959E8C9895988C9A959A8A98939811
:104F50000401010EA26FA56F0401D66B0E01006F54
:104F60000401AB6FB06BAC6BAD6BAE6BAF6BB16B89
:104F70009380F19EB26F1200D9CFE6FFE1CFD9FF47
:104F8000030EE126DF6A010EDB6A020EDB6AE66AC7
:104F9000D9CFE6FFDACFE6FF010EE66E13EC1AF08A
:104FA000E552E552E552E552E66AD950010FE66E48
:104FB000000EDA20E66E030EE66E13EC1AF0E552F0
:104FC000E552E552E5522C5001E014D1DF0446E1F0
:104FD000D950010FE96EDACFEAFFEE50ED1008E18B
:104FE0000E01006B0401D66B01017B6B7C6BEFD073
:104FF000D950010FE96EDACFEAFF010EEE180FE18A
:10500000ED500DE10401010ED66F0E01006B93927D
:1050100001015A0501E0DBD0020E5A6FD8D004011D
:10502000D66B9392B3CEE6FFB4CEE6FF040EE66EE7
:10503000B1CEE6FFB2CEE6FF010EE66E1FEC36F013
:10504000496E060EE15E4950000EE66EE66A010EFC
:10505000E66E0EDBE552E552E552B9D0020EDF5C9A
:1050600015E1D950010FE96EDACFEAFFEE50ED10ED
:105070000AE10401010EA56F959E959A9492959868
:105080009690959CA4D00401A56BA1D0040EDF5C82
:1050900007E1010EDBCFB1FE020EDBCFB2FE97D0EF
:1050A000050EDF5C07E1010EDBCFAFFE020EDBCFAA
:1050B000B0FE8DD0060EDF5C1CE1D950010FE96E09
:1050C000DACFEAFF720ED880EE542E0EED540AE2CB
:1050D000720EF36E010EF3CFDBFF2E0EF36E020E97
:1050E000F3CFDBFF010EDBCFA9F4020EDBCFAAF476
:1050F0006ED0070EDF5C1CE1D950010FE96EDACFEC
:10510000EAFF720ED880EE542E0EED540AE2720EB3
:10511000F36E010EF3CFDBFF2E0EF36E020EF3CF14
:10512000DBFF010EDBCFA7F4020EDBCFA8F44FD0DC
:10513000080EDF5C16E1D950010FE96EDACFEAFF05
:10514000180ED880EE54000EED5407E2180EF36EE0
:10515000010EF3CFDBFF020EDB6A010EDBCFABFEED
:1051600036D0090EDF5C16E1D950010FE96EDACFB7
:10517000EAFF060ED880EE54000EED5407E2060E4C
:10518000F36E010EF3CFDBFF020EDB6A010EDBCF05
:10519000ACFE1DD00A0EDF5C07E1010EDBCFB3FED3
:1051A000020EDBCFB4FE0DD00B0EDF5C07E1010E6B
:1051B000DBCFB3FE020EDBCFB4FE09D00C0EDF5CFA
:1051C00006E1010EDBCFB5FE020EDBCFB6FE0D0E03
:1051D000DF5C0EE1D950010FE96EDACFEAFFEE5045
:1051E000ED1004E00401010EB26F02D00401B26BB5
:1051F000F1EC11F0030EE15C02E2E16AE552E16ECE
:10520000E552E7CFD9FF1200D9CFE6FFE1CFD9FFB2
:105210000A0EE126020EDB6A030EDB6A040EDB6A6D
:10522000050EDB6A060EDB6A070EDB6A080EDB6A18
:10523000090EDB6AE66AD9CFE6FFDACFE6FF030E96
:10524000E66E13EC1AF0E552E552E552E552E66AD5
:10525000D950020FE66E000EDA20E66E020EE66E00
:1052600013EC1AF0E552E552E552E552010EE66EF6
:10527000D950040FE66E000EDA20E66E020EE66EDE
:1052800013EC1AF0E552E552E552E5522C5023E1B9
:10529000080EDBCFE6FF090EDBCFE6FF060EDBCF05
:1052A000E6FF070EDBCFE6FF040EDBCFE6FF050EC1
:1052B000DBCFE6FF020EDBCFE6FF030EDBCFE6FF20
:1052C000DECFE6FFDDCFE6FF10D8496E0A0EE15EC5
:1052D0004950F1EC11F00A0EE15C02E2E16AE5529C
:1052E000E16EE552E7CFD9FF1200D9CFE6FFE1CF5B
:1052F000D9FF1D50FEE1D950FB0FE96EFF0EDA20F9
:10530000EA6EEE50ED102EE1D950F90FE96EFF0E66
:10531000DA20EA6EEE50ED1025E1D950F70FE96E74
:10532000FF0EDA20EA6EEE50ED101CE1D950F50FB9
:10533000E96EFF0EDA20EA6EEE50ED1013E1040183
:10534000020E996F190E3D6E3E6AFD0EDBCF42F0E4
:10535000FE0EDBCF43F02EEC39F03BC09AF43CC09C
:105360009BF4EBD0010E04019A6F9B6B986B8D90B0
:105370008C9CFB0EDBCF49F0FC0EDBCF4AF0800E9D
:105380004A1413E0020E9811986F3D683E68FB0EB8
:10539000DBCF42F0FC0EDBCF43F001EC39F0FB0E2B
:1053A0003BC0DBFFFC0E3CC0DBFFF90EDBCF49F05E
:1053B000FA0EDBCF4AF00001800E4A1414E0080E0A
:1053C00004019811986F3D683E68F90EDBCF42F0FA
:1053D000FA0EDBCF43F001EC39F0F90E3BC0DBFFF6
:1053E000FA0E3CC0DBFFFD0EDBCF4DF0FE0EDBCF37
:1053F0004EF04F6A506A190E406E416A426A436A23
:105400004DC03BF04EC03CF04FC03DF050C03EF0B0
:10541000D6EC39F037C04DF038C04EF039C04FF0FF
:105420003AC050F0FB0EDBCF49F0FC0EDBCF4AF068
:105430004B6A4C6A4AAE02D04B684C680F0ED8904B
:1054400049364A364B364C36E806F9E149C03BF05E
:105450004AC03CF04BC03DF04CC03EF04DC040F067
:105460004EC041F04FC042F050C043F034EC3AF02F
:105470003BC088F43CC089F4010E04018827000E6B
:105480008923FB0EDBCF90F4FC0EDBCF91F4FD0EF5
:10549000DBCF4DF0FE0EDBCF4EF04F6A506A190E97
:1054A000406E416A426A436A4DC03BF04EC03CF0D8
:1054B0004FC03DF050C03EF0D6EC39F037C04DF053
:1054C00038C04EF039C04FF03AC050F0F90EDBCF83
:1054D00049F0FA0EDBCF4AF04B6A4C6A4AAE02D072
:1054E0004B684C680F0ED89049364A364B364C36CE
:1054F000E806F9E149C03BF04AC03CF04BC03DF042
:105500004CC03EF04DC040F04EC041F04FC042F0A4
:1055100050C043F034EC3AF03BC08AF43CC08BF40A
:10552000010E04018A27000E8B23F90EDBCF92F4C3
:10553000FA0EDBCF93F4010E996F010E1D6EE5524A
:10554000E7CFD9FF1200ABC449F04A6A49BE4A68A6
:1055500049C0E6FF4AC0E6FF280E4B6E6D0E4C6E4A
:105560004D6A4BC0E6FFE66E4DC0E6FFB5EC38F085
:105570004E6E050EE15E4E50F1EF11F0D9CFE6FF11
:10558000E1CFD9FF020EE126F40EDE6E010EDD6ED4
:10559000E66ED9CFE6FFDACFE6FF030EE66E13EC38
:1055A0001AF0E552E552E552E5522C5015E104019E
:1055B000AB0506E1DECFE6FFDDCFE6FFE66A06D00B
:1055C000DECFE6FFDDCFE6FF010EE66E51D8E552F5
:1055D000E552E552F1EC11F0020EE15C02E2E16A03
:1055E000E552E16EE552E7CFD9FF1200D9CFE6FFD1
:1055F000E1CFD9FF030EE126DF6A010EDB6A020E5E
:10560000DB6AE66AD9CFE6FFDACFE6FF010EE66E87
:1056100013EC1AF0E552E552E552E552010EE66E42
:10562000D950010FE66E000EDA20E66E030EE66E2C
:1056300013EC1AF0E552E552E552E5522C500EE11A
:10564000010EDBCFE6FF020EDBCFE6FFDFCFE6FF8A
:105650000FD8E552E552E552F1EC11F0030EE15C92
:1056600002E2E16AE552E16EE552E7CFD9FF1200AE
:10567000D9CFE6FFE1CFD9FF1D50FEE1FE0EDB04DE
:1056800003E10401030E02D00401040E996F190E08
:105690003D6E3E6AFC0EDBCF42F0FD0EDBCF43F0E9
:1056A0002EEC39F03BC09AF43CC09BF4010E1D6E09
:1056B000E552E7CFD9FF1200D9CFE6FFE1CFD9FFFE
:1056C000050EE126E66AD9CFE6FFDACFE6FF010E46
:1056D000E66E13EC1AF0E552E552E552E552E76E3C
:1056E000040EE7CFDBFFDB502FE12C5057E1040124
:1056F000A55124E0DF5000081FE28D90DF0403E194
:105700008D848D82898C020EDF5C03E18D848D8215
:10571000899C030EDF5C03E18D948D82899C040ECD
:10572000DF5C03E18D848D92899C050EDF5C0CE1CA
:105730008D948D92899C08D08D8006D0DF50000812
:1057400002E28D9001D08D80010EE66ED950010FDE
:10575000E66E000EDA20E66E010EE66E13EC1AF02D
:10576000E552E552E552E552E76E040EE7CFDBFF66
:10577000DB5012E12C5012E10401A55106E0010EAC
:10578000DB50000806E38C8C07D0010EDB500008CC
:1057900002E28C9C01D08C8CF1EC11F0050EE15CE6
:1057A00002E2E16AE552E16EE552E7CFD9FF12006D
:1057B000FE0E0401AC5DFF0EAD59FF0EAE59FF0E9B
:1057C000AF5905E2AC2B000EAD23AE23AF23F1EFB2
:1057D00011F00401AC51AD11AE11AF1105E0AC07F1
:1057E000000EAD5BAE5BAF5BF1EF11F0D9CFE6FF22
:1057F000E1CFD9FF050EE126E66AD9CFE6FFDACF81
:10580000E6FF070EE66E13EC1AF0E552E552E5529C
:10581000E552E76E040EE7CFDBFFDB500BE1DFCF95
:10582000ACF4010EDBCFADF4020EDBCFAEF4030E11
:10583000DBCFAFF4F1EC11F0050EE15C02E2E16ABE
:10584000E552E16EE552E7CFD9FF1200ACC4E6FFA6
:10585000ADC4E6FFAEC4E6FFAFC4E6FF1F0E496E5F
:105860006D0E4A6E4B6A49C0E6FFE66E4BC0E6FF1E
:10587000B5EC38F04C6E070EE15E4C50F1EF11F0D4
:10588000E66AB00EE66E040EE66E010EE66E13ECEE
:105890001AF0E552E552E552E5522C5001E01200B3
:1058A000F1EF11F0B0C449F04A6A49BE4A6849C0F4
:1058B000E6FF4AC0E6FF180E4B6E6D0E4C6E4D6A49
:1058C0004BC0E6FFE66E4DC0E6FFB5EC38F04E6E1D
:1058D000050EE15E4E50F1EF11F0B1C449F04A6A95
:1058E00049BE4A6849C0E6FF4AC0E6FF120E4B6E49
:1058F0006D0E4C6E4D6A4BC0E6FFE66E4DC0E6FF86
:10590000B5EC38F04E6E050EE15E4E500401B16B01
:10591000F1EF11F0D9CFE6FFE1CFD9FF040EE12678
:10592000DE6ADD6A020EDB6A030EDB6AC26AA40E5F
:10593000C16E9E9C9F9CC28004010A0EB36FB3513E
:10594000FEE1C282C2B2FED7C4504C6E4B6AC35055
:105950004B24496E000E4C2049C0DEFFDD6E2D0E3B
:10596000C26E04010A0EB36FB351FEE1C282C2B22D
:10597000FED7C4504C6E4B6AC35000014B24496E95
:10598000000E4C204A6E020E49C0DBFF030E4AC0D7
:10599000DBFF020EDBCFE6FF030EDBCFE6FFDECF41
:1059A000E6FFDDCFE6FF060E496E6D0E4A6E4B6ACE
:1059B00049C0E6FFE66E4BC0E6FFB5EC38F04C6E32
:1059C000070EE15E4C50F1EC11F0040EE15C02E2D6
:0E59D000E16AE552E16EE552E7CFD9FF120021
:0259DE002BECB0
:1059E00032F0FB0EDBCFF3FFDB06F35000090AE0D9
:1059F00079EC32F0FA0EE4EC32F0F3E14A1CF1E11A
:105A0000010E01D0000E5AEF32F02BEC32F03B0EBB
:105A1000E12402E3E168E652E16E010EDB6A020E68
:105A2000DB6AF90EDBCFF6FFFA0EDBCFF7FFFB0EDA
:105A3000DBCFF8FF0800F550DF6EDF5002E17EEFAC
:105A400031F0250EDF5C02E071EF31F0030EDB6A0E
:105A5000040EDB6A050EDB6A060EDB6A070EDB6AE4
:105A600093EC31F02D0EDF5C0CE02B0EDF5C09E0D7
:105A7000200EDF5C06E0230EDF5C03E0300EDF5C0F
:105A80001AE1DF50300A14E0130A0FE0030A0AE0BB
:105A90000B0A05E0060AE4E1030EDB80E1D7030E02
:105AA000DB82DED7030EDB84DBD7030EDB86D8D7A1
:105AB000030EDB88D5D72A0EDF5C1BE18FEC31F0BB
:105AC000DDEC31F010E0030EDB803D683E68130E24
:105AD000DBCF42F0140EDBCF43F001EC39F0040EC3
:105AE0003BC0DBFF03D0130EC6EC31F093EC31F07A
:105AF0000BD0090EDB6A34EC32F003E0A8EC32F094
:105B0000FAD7090EC6EC31F0030EDBB0DB982E0E8F
:105B1000DF5C1BE193EC31F02A0EDF5C0BE18FECD4
:105B200031F0DDEC31F003E1130E18EC32F093ECC0
:105B300031F00BD0090EDB6A34EC32F003E0A8EC54
:105B400032F0FAD7090E18EC32F0680EDF5C07E18C
:105B500093EC31F0680EDF5C1DE1030E18D0740E7B
:105B6000DF5C17E07A0EDF5C14E0480EDF5C06E0D5
:105B7000540EDF5C03E05A0EDF5C02E1020E07D038
:105B80006C0EDF5C03E06A0EDF5C04E1010E6BEC7F
:105B900032F0C9DBDF506E0A01E17FD31E0A01E15A
:105BA00092D1200A01E18FD13F0A01E149D11A0ABD
:105BB00001E146D10D0A01E143D1200A01E140D1C2
:105BC0003A0A01E13DD1200A01E13AD1260A01E178
:105BD00035D10D0A01E132D11A0A01E1D9D0200AEA
:105BE0004AE0300A1FE0460A0EE0250A01E083D3AE
:105BF000D950F90FE96EFF0EDA20EA6E010EEE5E63
:105C0000000EEE5AEE5A79EC32F0250EE66E95DB78
:105C100003E14A1C01E169D375EC32F001E26BD378
:105C2000DB2A69D3080EDB6A040EDB50010806E2AA
:105C3000040EDB043DEC32F0DB508BDB080EDB5056
:105C400009E0030EDB50010B05E172DB01E04DD3EF
:105C5000080EDB6A64DBEFCFDFFFEDEC32F003E12F
:105C60004A1C01E142D375EC32F001E3DB2A60DB30
:105C700001E141D33AD3070EDB5002080FE1B9EC42
:105C800032F0030E80EC32F00E0EEECFDBFF0F0E83
:105C9000EECFDBFF100EEECFDBFF20D0F70EDBCF19
:105CA0004CF0F80EDBCF4DF0020E4C5E000E4D5A5C
:105CB000F70E4CC0DBFFF80E4DC0DBFF4CC0E9FF18
:105CC0004DC0EAFF70EC32F04B6A0E0E49C0DBFFAC
:105CD0000F0E4AC0DBFF100E4BC0DBFF0E0EDBCFFA
:105CE000E6FF0F0EDBCFE6FF100EDBCFE6FF90ECFA
:105CF00038F0E552E552E552130E3CC0DBFF140EBE
:105D00003DC0DBFF060EDB5005E0130EB4EC32F0B5
:105D100001E26ADBD8EC32F002E2130E37DB9BECD7
:105D200032F006E0040EB4EC32F002E2050E2EDB97
:105D3000030EDBB005D0FCDA01E0D7D2080EDB6A37
:105D4000090EDB6A0E0EDBCFF6FF0F0EDBCFF7FF7F
:105D5000100EDBCFF8FF0800F550DF6EDF5014E0C7
:105D6000DEEC32F011E2EDEC32F003E14A1C01E12D
:105D7000BCD2BBDB01E3DB2A090EDB2AD9500E0FB4
:105D8000E96E000ECBDBE7D7D3DA01E1B4D2ADD2B6
:105D9000C6DA110EEECFDBFF120EEDCFDBFF110ED8
:105DA000DBCFE6FF120EDBCFE6FF82EC38F0E552E8
:105DB000E552130EF3CFDBFF140EF4CFDBFF060E1C
:105DC000DB5004E0130ED0DB01E20EDBD8EC32F046
:105DD00002E2130EDBDAAFDB05E0040EC5DB02E204
:105DE000050ED4DA030EDBB005D0A2DA01E07DD2D5
:105DF000080EDB6A090EDB6A110EDBCFE9FF120E1B
:105E0000DBCFEAFFEFCFDFFFDF5014E0D7DB12E29A
:105E1000E4DB03E14A1C01E168D267DB01E3DB2A32
:105E2000090EDB2A110EDB2ADBCFE9FF120EE8E3B5
:105E3000DB2AE6D77DDA01E15ED257D2030EDB8E94
:105E4000070EDB0410E195DB040E5ADB0A0EEECFE1
:105E5000DBFF0B0EEECFDBFF0C0EEECFDBFF0D0EEC
:105E6000EECFDBFF6CD0070EDB5003082CE1030EF6
:105E7000DBAE0DD0B2DA020E76DAEFCF49F04A6A25
:105E80004B6A4C6A49AE39D04A684B6835D0F70E38
:105E9000DBCF4AF0F80EDBCF4BF0020E4A5E000E6D
:105EA0004B5AF70E4AC0DBFFF80E4BC0DBFF4AC06F
:105EB000E9FF4BC0EAFFEFCF49F00A0E49C0DBFF14
:105EC0000B0EDB6A38D0070EDB50020809E1030E27
:105ED000DBAE04D059DB4BAE10D00ED055DB0DD06D
:105EE000030EDBAE12D079DA020E3DDAF9DA4B6A34
:105EF0004C6A4AAE02D04B684C68E2DA0C0E4BC0DA
:105F0000DBFF0D0E4CC0DBFF1AD0F70EDBCF4BF0E2
:105F1000F80EDBCF4CF0020E4B5E000E4C5AF70E23
:105F20004BC0DBFFF80E4CC0DBFF4BC0E9FF4CC0A1
:105F3000EAFFD6DAC5DA0C0EDB6A0D0EDB6A060E56
:105F4000DB5005E1010EF36E050EF3CFDBFF150EFE
:105F5000DB6A160EDB6AD950370F496E000EDA2065
:105F60004A6E390E49C0DBFF3A0E4AC0DBFF380EDD
:105F7000DB6A080EDB6A0A0EAEDADF50780A12E03E
:105F8000200A10E0280A0CE0200A0AE03F0A06E096
:105F90000D0A02E0200A08E1020E05D0080E03D027
:105FA000080EDF26100E97DA030EDBBE02D0DB925E
:105FB000DB94DB50800B24E08ADAD890030EEB50A0
:105FC000000A08E6000EEE5C000EEE58000EEE58D9
:105FD000000EEE5815E213DA4068416842684368E3
:105FE000D6EC39F00A0E37C0DBFF0B0E38C0DBFFF2
:105FF0000C0E39C0DBFF0D0E3AC0DBFF2D0E08D0B2
:10600000030EDBA202D02B0E03D0DBA408D0200E9F
:10601000F36E170EF3CFDBFF150EDB2A02D0170E3F
:10602000DB6A050EDB5003E1B7D901E189D0340EFC
:10603000496E750E4A6E000E4B6E070EDBCF4CF0AC
:106040004D6A4E6A4F6A4CC040F04DC041F04EC0A0
:1060500042F04FC043F0D3D934EC3AF049503724E2
:10606000F36E4A503820F46E4B503920F86EF4CF5E
:10607000F7FFF3CFF6FF0800090EF5CFDBFF580E50
:10608000DF5C0FE1610EF36E090E7BD90AE3200E8F
:10609000496E090EDBCFE7FF4950E75E090EE7CFF7
:1060A000DBFF070EDBCF49F04A6A4B6A4C6A0FDA16
:1060B00049C040F04AC041F04BC042F04CC043F0F0
:1060C000EECF3BF0EECF3CF0EECF3DF0EFCF3EF029
:1060D00034EC3AF03EC0EDFF3DC0EDFF3CC0EDFFBB
:1060E0003BC0EFFF390EDBCFE9FFDB063A0EDBCF1B
:1060F000EAFF01E2DB06090EDBCFEFFF150EDB2A1C
:106100004BD995E1030EDBA61DD06F0EDF5C06E1D7
:10611000C1D918E3150EDB285BDA14D0780EDF5CEA
:1061200009E0580EDF5C06E0620EDF5C03E0420E21
:10613000DF5C08E1020EF36E160EF3CFDBFF02D038
:10614000150EDB6A030EDB50100B0EE0040EDBCFE6
:1061500049F0050EDB50D880495406E2060EDB50AC
:1061600003E1040EDB5034DA95D90AE2050EDBCFE9
:10617000E7FF150EDB50E75E050EE7CFDBFF02D031
:10618000050EDB6A040EDBCF49F0160E45D9D88028
:10619000495414E2160EDBCFE6FF150EDBCFE6FF07
:1061A000040EDBCFE6FF050EDB50E552E75CE5525F
:1061B000D880E754E552D880E7545FD9030EDB500E
:1061C000010B0BE1080EDB5008E0B2D801E08DD0E6
:1061D000080EDB50BED8080EDB6A170EDB5007E056
:1061E00088D9170EF1D903E14A1C01E17ED0160EC1
:1061F000DB5016E07ED9300EE66E9FD802E14A1CD5
:1062000074E077D9DFCFE6FF94EC39F0E552E55240
:10621000E552F4CF4AF00001F31C02E14A1C65E0AC
:10622000050EDBCF49F0160EDB50D880495409E249
:10623000050EDBCFE7FF160EDB50E75E050EE7CF5E
:10624000DBFF300EE66E050ECBD94FE1390EDB2AAF
:10625000DBCFE9FF3A0E01E3DB2ADBCFEAFF090ED1
:10626000EFCFDBFFDB500EE044D9090EADD902E1E0
:106270004A1C3BE0390EDB2ADBCFE9FF3A0EEDE3A7
:10628000DB2AEBD755D831E1160EDBCFE6FF080E3F
:10629000C3D8E552E7245DD82ED0070EDB50030AA1
:1062A0001CE0010A14E0030A07E07BD9DBCFEEFF14
:1062B000020EDBCFEDFF1FD0F5D84E6A4CAE02D0F8
:1062C0004D684E682CD8BCD84EC0EEFF14D0EAD82A
:1062D0004CBE4D6824D8B4D80ED063D9DBCFEFFFC5
:1062E0000AD07BD905E14A1C03E1F368F46810D0B9
:1062F000FCD801E3DB2A79D91AEF2DF0010EDBCFB0
:1063000049F0020EDBCF4AF049C0F3FF4AC0F4FF68
:106310003B0EE15C02E2E16AE552E16ECBD029D9A5
:10632000020E80EF32F061D90800F550DF6E1200E6
:10633000200EE66E080EF0EF32F094EC39F0E552E4
:10634000E552E552F3CF49F0F4CF4AF00001F31CD7
:106350001200496E4A6AD950010F4DD94950EE26B4
:106360004A50ED2212004D5E000E4E5AF70E4DC0FF
:10637000DBFFF80E4EC0DBFF4DC0E9FF4EC0EAFF69
:106380001200DBCFF4FFF350F45C1200DB50E76E39
:10639000040EE7CFDBFF12000A0EDBCF49F00B0E35
:1063A000DBCF4AF00C0EDBCF4BF00D0EDBCF4CF009
:1063B00049504A104B104C101200130EEECFDBFF69
:1063C000140EEDCFDBFF130EDBCF49F0140EDBCF45
:1063D0004AF00001800E4A141200F70EDBCF4DF098
:1063E000F80EDBCF4EF01200050EDB50E66ED950F2
:1063F000130F01D9E552E750EE6EED6A12000A0E56
:10640000DBCF3BF00B0EDBCF3CF00C0EDBCF3DF0D7
:106410000D0EDBCF3EF01200DBCFE6FF150EDBCF1B
:10642000E6FF050EDB50E552E724E552E7241200B3
:10643000DB50CED8010EF36E060EF3CFDBFF120059
:10644000EE50EFCFEAFFE96E4BC0EEFF4CC0EEFF1F
:106450004DC0EEFF1200D9CFE6FFDACFE6FFE1CF65
:10646000D9FFE2CFDAFF1200DFCFE6FFE66A22ECC7
:106470003AF0E552E552F3501200E76E080EE7CF0E
:10648000DBFF1200EECF49F0EECF4AF0EFCF4BF03A
:106490004C6A1200050EDBCF49F0150EDB50D88098
:1064A00049541200010EDBCF4BF0020EDBCF4CF053
:1064B0004D6A1200E552E5CFDAFFE7CFD9FF1200AF
:1064C0000A0E49C0DBFF0B0E4AC0DBFF1200D95099
:1064D0000A0FFBEF32F0F36E070EF3CFDBFF120073
:1064E000EECF49F0EFCF4AF01200010EDB2A020E88
:1064F0001200FC0EDBCFE6FFFD0EDBCFE6FF120045
:10650000495E000E4A5AF70E49C0DBFFF80E4AC03A
:10651000DBFF49C0E9FF4AC0EAFF1200DA20EA6E59
:10652000EF2AEECFF6FF000EEF22EECFF7FFEF22BD
:10653000EECFF8FF1200040EDBCFE6FF130EDB50A8
:10654000E552E75C9ADFDB5004DF060EDB501200F9
:10655000090EDB500A0DF350DF24D00FE76E090E51
:10656000E7CFDBFF93EF31F0DB50F36E050EC1EFA9
:1065700031F0F70EDBCF49F0F80EDBCF4AF0120016
:10658000DFCFE6FF9DEF31F028DF030EECDE42EFB8
:1065900032F0EFEC2CF0E552E552E552E5520009FD
:1065A0001200BDDEEE50EFCFEAFFE96E010E1200E1
:1065B000130EDB50F36E040EC1EF31F0040EDB500E
:1065C000F36E090EC1EF31F0DBCFE6FF9DEF31F046
:1065D000E76E050EE7CFDBFF12008BDFC0EF32F076
:1065E000DBCFE6FF86DFC9EF32F0D950F90FE96E55
:1065F000FF0E8EEF32F0E96E000EDA20EA6E120026
:10660000040140511F0B010801E012004051600BD2
:10661000E842E842E842E842E842010801E01200AC
:10662000445103E0440501E012004151220A31E0E7
:10663000030A24E0010A15E0210A0DE0010A01E045
:1066400012000501A00EC16F050EC26F080EC46FC7
:10665000C56BC38121D00501A00EC16F050EC26FAD
:106660001BD046C4C9F547C4CAF50501880EC66FDC
:10667000050EC76FCB6BCC6BC88F12000501880E5F
:10668000C16F050EC26F070EC46FC56BC10EC36F1D
:10669000120042C49BF50501C38F12000501886BEF
:1066A0004B0E896F8A6B8B6B8C6B8D6B080E8E6FAC
:1066B000906B8F6B1A0EE66E020EE66E6EEC24F097
:1066C000E552E5521E0EE66E030EE66E6EEC24F009
:1066D000E552E552400EE66E080EE66E050EE66ED9
:1066E000E66A030EE66E12EC25F0496E050EE15ED9
:1066F0004950F3CF97F5F4CF98F50501996B9A6B54
:106700001200D9CFE6FFE1CFD9FF05018F6B97517A
:10671000981102E1000E08D097C5E9FF98C5EAFF7D
:10672000EF50800B01E0010E000945E1FC0EDBCFCC
:1067300049F097C5E9FF98C5EAFFEE52EF50D880BF
:10674000495408E297C5E9FF98C5EAFFEE52FC0EEE
:10675000EFCFDBFF8F6BFC0EDB508F5D19E28F51AB
:10676000EA6A080FE96E050EEA22EF50E66E8F51D5
:10677000E76EFD0EDBCFE9FFFE0EDBCFEAFFE75051
:10678000E926000EEA22E552E750EF6E8F2BE3D7A1
:10679000400EE66E080EE66E050EE66EE66A030E25
:1067A000E66E12EC25F0496E050EE15E4950F3CF1E
:1067B00097F5F4CF98F505018F51E552E7CFD9FF52
:1067C0001200D9CFE6FFE1CFD9FF050190510CE1CE
:1067D000FD0EDBCF91F5FE0EDBCF92F5FC0EDBCF8D
:1067E00095F5010E966F906FE552E7CFD9FF120035
:1067F000D9CFE6FFE1CFD9FF030EE1260501905185
:106800002DE1DF6AFD0EDBCF3DF0FE0EDBCF3EF06B
:10681000DE523DC0DEFF3EC0DDFFDD52DF2ADF502D
:10682000496E4A6AFF0E491802E14A500BE0010E18
:10683000DBCFE9FFDB2A020EDBCFEAFF01E3DB2A35
:10684000EF50ECE1FD0EDBCF91F5FE0EDBCF92F5C4
:10685000DFCF95F50501010E966F906F030EE15C99
:1068600002E2E16AE552E16EE552E7CFD9FF12009C
:10687000D9CFE6FFE1CFD9FF030EE1260501905104
:106880002EE1DF6AFD0EDBCF3DF0FE0EDBCF3EF0EA
:10689000DE523DC0DEFF3EC0DDFFDD52DF2ADF50AD
:1068A000496E4A6AFF0E491802E14A500CE0010E97
:1068B000DBCFF6FFDB2A020EDBCFF7FF01E3DB2A9B
:1068C0000800F550EBE1FD0EDBCF91F5FE0EDBCFBE
:1068D00092F5DFCF95F50501966B010E906F030ED3
:1068E000E15C02E2E16AE552E16EE552E7CFD9FFF1
:1068F0001200D9CFE6FFE1CFD9FF020EE126050154
:1069000099519A1102E1000E08D099C5E9FF9AC584
:10691000EAFFEF50800B01E0010E000901E084D096
:10692000030E905D01E1906B905101E17DD0020E6C
:10693000905D16E1E66A000EE66EE66A010EE66E0E
:10694000030EE66E12EC25F0496E050EE15E49502D
:10695000F3CF99F5F4CF9AF50501030E906F64D04B
:10696000900562E1400E496E4A6A9551495C000EFD
:106970004A5803E2400EDF6E02D095C5DFFFDF50BC
:10698000955D956F480E936F050E946F010EDFCFE6
:10699000DBFF965116E1010EDB5028E091C5F6FFB2
:1069A00092C5F7FF0800F55093C5E9FF94C5EAFFCB
:1069B000EF6E932B000E9423912B9223010EDB0696
:1069C000EAD7010EDB5012E091C5E9FF92C5EAFF5C
:1069D000EF5093C5E9FF94C5EAFFEF6E932B000ECD
:1069E0009423912B9223010EDB06EBD705019551E1
:1069F00007E1400EDF5C02E1020E01D0030E906F52
:106A0000DFCFE6FF480EE66E050EE66E010EE66E7F
:106A1000030EE66E12EC25F0496E050EE15E49505C
:106A2000F3CF99F5F4CF9AF5020EE15C02E2E16A48
:0C6A3000E552E16EE552E7CFD9FF1200FD
:046A3C00D9CFE6FFC9
:106A4000E1CFD9FFE6520E01006B016BAA6BDF6A42
:106A5000180EDF5C2AE2EA6ADF34FE0BEA36E96EE2
:106A6000020EE9260E0EEA22EE6AED6ADF50EA6AAD
:106A7000320FE96E0E0EEA22EF6AEA6ADF34FE0B8D
:106A8000EA36E96E4A0EE9260E0EEA22EE6AED6A51
:106A9000EA6ADF34FE0BEA36E96E7A0EE9260E0E5C
:106AA000EA22EE6AED6ADF2AD3D70E01C60EAD6F79
:106AB0000E0EAE6F3F0E79140009796ECF0E791469
:106AC0000009796E79827B6A7A6A79900F01528126
:106AD0005293F00EB4140909B46E0E01070EAB6F99
:106AE000030EAC6FE00EB16F2E0EB26F800EAF6F63
:106AF0003E0EB06F0401D66B93920E01010E006F33
:106B0000900EB36F010EB46F900EB56F010EB66F9D
:106B1000B3CEE6FFB4CEE6FF040EE66EB1CEE6FFDE
:106B2000B2CEE6FF010EE66E8AD8496E060EE15E31
:106B30004950000EE66EE66A010EE66E38EC2BF068
:106B4000E552E552E552E552E552E7CFD9FF120092
:106B5000D9CFE6FFE1CFD9FF050EE126DF6A010EAE
:106B6000DB6A020EDB6A030EDB6A040EDB6AE66A8E
:106B7000D9CFE6FFDACFE6FF010EE66E13EC1AF08E
:106B8000E552E552E552E552010EE66ED950010F8D
:106B9000E66E000EDA20E66E030EE66E13EC1AF0D7
:106BA000E552E552E552E552010EE66ED950030F6B
:106BB000E66E000EDA20E66E010EE66E13EC1AF0B9
:106BC000E552E552E552E552010EE66ED950040F4A
:106BD000E66E000EDA20E66E030EE66E13EC1AF097
:106BE000E552E552E552E5522C501FE1DF501808FE
:106BF00004E3030EDB50180802E22C8C16D0040EBE
:106C0000DBCFE6FFE66A030EDBCFE6FF010EDBCF4C
:106C1000E6FF020EDBCFE6FFDFCFE6FF10D8496EBE
:106C2000060EE15E4950F1EC11F0050EE15C02E266
:106C3000E16AE552E16EE552E7CFD9FF1200D9CF04
:106C4000E6FFE1CFD9FFFE0EDB5003E10E01006B42
:106C500056D0FE0EDB50180852E3FB0EDB5018082E
:106C60004EE30E01010E006FFE0EDB04E96EEA6AD0
:106C7000D890E936EA367A0EE9260E0EEA22F90EA7
:106C8000DBCFEEFFFA0EDBCFEDFFFE0EDB04E96E8D
:106C9000EA6AD890E936EA364A0EE9260E0EEA226A
:106CA000FC0EDBCFEEFFFD0EDBCFEDFFFE0EDB04B7
:106CB000EA6A320FE96E0E0EEA22FB0EDBCFEFFF1F
:106CC000FE0EDB04E96EEA6AD890E936EA36020E77
:106CD000E9260E0EEA22EE50ED1011E1FE0EDB0465
:106CE000E96EEA6AD890E936EA36020EE9260E0E17
:106CF000EA22FC0EDBCFEEFFFD0EDBCFEDFFE5520F
:066D0000E7CFD9FF1200ED
:0A6D0600253034692C253034690D66
:106D10000A002531690D0A00253033690D0A002566
:106D20003031306C750D0A0025640A0D0053746112
:106D30007475733D25690D0A002135204572723A3C
:106D4000204E65656420636F6D6D61206E6578749B
:106D50002C20666F756E643A20272563270D0A0084
:106D6000506172616D383D25630D0A00506172619A
:106D70006D373D25630D0A00506172616D363D250A
:106D80006C750D0A00506172616D353D256C640DA6
:106D90000A00506172616D343D25750D0A00506125
:106DA00072616D333D25640D0A00506172616D3270
:106DB0003D25640D0A00506172616D313D25640D01
:106DC0000A0050492C2531750D0A004D522C2530F2
:106DD00033750D0A002C25303475004100492C25EF
:106DE0003033692C253033692C253033692C25301C
:106DF00033692C253033690D0A0021382045727221
:106E00003A20556E6B6E6F776E20636F6D6D616E9D
:106E1000642027256325633A253258253258270DEB
:106E20000A002138204572723A20556E6B6E6F77DA
:106E30006E20636F6D6D616E64202725633A253285
:106E400058270D0A002137204572723A2045787480
:106E50007261207061726D617465720D0A00213675
:106E6000204572723A20496E76616C6964207061C7
:106E700072616D7465722076616C75650D0A002112
:106E800034204572723A204D697373696E672070C1
:106E90006172616D657465722873290D0A00213372
:106EA000204572723A2052582042756666657220FB
:106EB0006F76657272756E0D0A002132204572720E
:106EC0003A20545820427566666572206F76657266
:106ED00072756E0D0A002131204572723A204361AD
:106EE0006E27742073746570207468617420666105
:106EF00073740D0A002130200D0A0020080025734C
:0D6F0000001B5B421B5B314B1B5B304700ED
:026F0E0005D8A4
:106F1000D4EC1DF00BEC0DF0FBD7D9CFE6FFE1CFA1
:106F2000D9FF020EE1260F0148694969600ED36E50
:106F30009B8C580EDE6E020EDD6EDFCF49F0DF0651
:106F4000010EDBCF4AF001E2DB0649504A10F5E1C1
:106F5000948E4AEC0CF066EC1DF0020EE15C02E24D
:106F6000E16AE552E16EE552E7CFD9FF1200120067
:106F700012001200120000EF33F012004EEF33F057
:106F800065840101080EFD6F070EFE6FFD07000E00
:106F9000FE5BFD51FE11FAE165941200D9CFE6FFC8
:106FA000E1CFD9FFFD0EDBCF3DF0FE0EDBCF3EF093
:106FB000720E3D1801E13E5033E0E8683D1802E1F1
:106FC0007F0E3E182BE0740E3D1801E13E5024E088
:106FD000750E3D1801E13E501DE0730E3D1801E1B4
:106FE0003E5016E0030E3D1801E13E500FE0020E48
:106FF0003D1801E13E5008E0010E3D1801E13E5010
:1070000001E010D0BBDF0FD0B8DF0DD0B4DF0BD064
:10701000B0DF09D0ACDF07D0ABDF05D0ABDF03D0EA
:10702000000001D000D0010E00D0E552E7CFD9FF1B
:0270300012004C
:0E7032002A0EF66E100EF76E000EF86E0501B7
:107040000900F550E36F0900F550E46F03E1E367D1
:1070500001D03DD00900F550DE6F0900F550DF6F1B
:107060000900F550E06F09000900F550E96E0900CC
:10707000F550EA6E090009000900F550E16F0900BA
:10708000F550E26F09000900F6CFE5F5F7CFE6F518
:10709000F8CFE7F5DEC5F6FFDFC5F7FFE0C5F8FF7F
:1070A0000501E15302E1E25307E00900F550EE6EFD
:1070B000E107F8E2E207F9D7E5C5F6FFE6C5F7FF15
:1070C000E7C5F8FF0501E307000EE45BBFD7120038
:1070D000FE0EE3CFE9FFFF0EE3CFEAFFE9CFF3FFB8
:1070E000EACFF4FFFB0EE35003E1FC0EE35009E0AE
:1070F000FB0EE30602E2FC0EE306FD0EE350EE6E2D
:10710000F1D71200FE0EE3CFE9FFFF0EE3CFEAFF57
:10711000F36AF46AEE5203E0F34AF42AFBD7120052
:10712000FF0EE3CFF8FFE552FF0EE3CFF7FFE55286
:10713000FF0EE3CFF6FFE552E66AE66AE66A09006B
:10714000F55209E0FD0EE32A05E1FE0EE32A02E115
:10715000FF0EE32AF4D7FD0EE3CF3CF0FE0EE3CFA3
:0A7160003DF0FF0EE3CF3EF01200F9
:06716A00D9CFE6FFDACFE9
:10717000E6FFE1CFD9FFE2CFDAFFE652E652E65270
:10718000E652D950FB0F496EFF0EDA204A6E49C015
:10719000DEFFDD6EDECFE6FFDDCFE6FFFB0EDBCFF1
:1071A000E6FFFC0EDBCFE6FFFD0EDBCFE6FFB7CE42
:1071B000E6FFB8CEE6FF05EC2DF0496E070EE15C68
:1071C00002E2E16AE552E16E4950020EF3CFDBFFC5
:1071D000030EF4CFDBFF020EDBCF49F0030EDBCF53
:1071E0004AF049C0F3FF4AC0F4FF040EE15C02E23A
:1071F000E16AE552E16EE552E5CFDAFFE7CFD9FF6C
:0272000012007A
:0E7202003EC048F03DC047F03D504202F4CF80
:107210003CF0F3CF3BF03E504302F4CF3EF0F3CFCF
:107220003DF04202F3503C26F4503D22E86A3E22F3
:1072300047504302F3503C26F4503D22E86A3E2278
:1072400043AE27EF39F047503D5E48503E5A48AEB6
:10725000000C42503D5E43503E5A000C3DC047F08A
:107260003D504202F4CF3CF0F3CF3BF03E5043029E
:10727000F4CF3EF0F3CF3DF04202F3503C26F45001
:107280003D22E86A3E2247504302F3503C26F45028
:087290003D22E86A3E22000CD9
:08729800120100020200004097
:1072A000D80492FD8201010200010902430002019B
:1072B00000C0320904000001020201000524001090
:1072C000010424020205240600010524010001072F
:1072D00005820308000209040100020A00000007F9
:1072E0000503024000000705830240000004030973
:1072F0000418035300630068006D0061006C007A9D
:1073000000480061007500730016034500690042E3
:10731000006F00740042006F00610072006400AAF8
:0773200072ED72F1720973B6
:08732800D9CFE6FFDACFE6FF42
:10733000E1CFD9FFE2CFDAFFFB0EDBCF49F0FC0E45
:10734000DBCF4AF00001800E4A141AE1FB0EDBCFBE
:10735000E9FFFC0EDBCFEAFFEECFF3FFEDCFF4FF4A
:10736000EE2A000EEF22F3CFE9FFF4CFEAFFFD0E85
:10737000DBCFEFFFEF504A6AF36E4AC0F4FF10D044
:10738000FB0EDB50FE0806E1FD0EDBCFE6FF8CECCA
:107390003AF005D0FD0EDBCFE6FFFEEC0EF0E55235
:0C73A000E552E5CFDAFFE7CFD9FF12007D
:0473AC003B50400210
:1073B000F3CF37F0F4CF38F04102F3503826000E07
:1073C000F420396E3B504202F3503926000EF4206F
:1073D0003A6E3B504302F3503A263C504002F35081
:1073E0003826F4503922000E3A223C504102F35024
:1073F0003926F4503A223C504202F3503A263D508E
:107400004002F3503926F4503A223D504102F350E5
:0C7410003A263E504002F3503A2612008B
:04741C00FF0EE1245A
:10742000E96EFF0EE220EA6EEDCFF4FFEFCFF3FF3F
:10743000F46607D0600EF36404D07B0EF36001D0D5
:10744000F39A1200F36AF46AFF0EE124E96EFF0E6C
:10745000E220EA6EED6607D02F0EEF6404D03A0EFC
:08746000EF6001D0F32A1200D5
:087468003A6A396A386A376A92
:10747000200EE76ED8903B363C363D363E363736EA
:10748000383639363A364050375C415038584250D9
:10749000395843503A5809E34050375E4150385A02
:1074A0004250395A43503A5A3B2AE72EE4D7120049
:1074B0004F4B0D0A000D0A004542427631322045FD
:1074C00042204669726D77617265205665727369F4
:0B74D0006F6E20322E302E320D0A00AD
:0474DC00C00EF36E7D
:1074E00000EE00F00E0E01D81200EA6002D0EE6A43
:0C74F000FCD7F350E9601200EE6AFCD7F4
:0474FC001DEE00F091
:107500002DEE00F0F86A369C19EC38F0A3EC3AF056
:0875100087EC37F0FBD71200F5
:08751800FF0EE350ADBA04D0F0
:10752000B06AAC8EAD8A949CADA2FED7AE6EF36EFF
:04753000F46A1200E7
:0C7534003031323334353637383961627B
:057540006364656600B4
:02754600120031
:02754800FEFF44
:06754A000000000000003B
:10755000000000000000000000000000000000002B
:10756000000000000000000000000000000000001B
:10757000000000000000000000000000000000000B
:1075800000000000000000000000000000000000FB
:1075900000000000000000000000000000000000EB
:0E75A0000000000000000000000000000000DD
:00000001FF
